:1000000016EF21F000000000ECEF1FF000000000F0
:100010000000000000000000E3EF20F0ADB202D0CD
:100020000000FCD7CAC4AEFF1200A8B202D0000084
:10003000FCD7CAC4A9FF12000B840BAE27EF00F057
:10004000010E036E026A016A006A0A360232FF0E6E
:100050001200026A016A006A086A036A000E12004E
:100060000B820BAE3AEF00F003680268016800688B
:100070000A360232FF0E12000AAE029E000E120075
:100080000CB082EF00F00CA228EF01F00E6A000E17
:10009000026499EF00F0F00E0214D8A464EF00F0AF
:1000A000023A01380F0B02260138F00B016E0038BE
:1000B0000F0B01260038F00B006E08380F0B0026DE
:1000C0000838F00B086E0E84D89002BE7DEF00F069
:1000D00008360036013602360E2A02BE7DEF00F0E9
:1000E00008360036013602360E2A02BE7DEF00F0D9
:1000F00008360036013602360E2A0E5003641EEF13
:1001000001F0035E0BBC08AE23EF01F0D880800E37
:1001100008640030000E002201220222D8A023EF42
:1001200001F0023201320032034A28EF01F023EFDE
:1001300001F001C002F000C001F008C000F0086A40
:10014000000E0E860264D0EF00F0F00E0214D8A468
:10015000B8EF00F0023A01380F0B02260138F00B1D
:10016000016E00380F0B01260038F00B006E0E8474
:10017000D89002BE7DEF00F00036013602360E2A1E
:1001800002BE7DEF00F00036013602360E2A02BEB6
:100190007DEF00F00036013602360E2A7DEF00F0CA
:1001A00001C002F000C001F0006A000E0E960E8839
:1001B0000264FDEF00F0F00E0214D8A4E8EF00F0A6
:1001C000023A01380F0B02260138F00B016E0E8443
:1001D000D89002BE7DEF00F0013602360E2A02BE34
:1001E0007DEF00F0013602360E2A02BE7DEF00F0F0
:1001F000013602360E2A7DEF00F001C002F0016ADE
:10020000000E0E8602642DEF01F0F00E0214D8A449
:100210000CEF01F0023A0E84D89002BE7DEF00F0A0
:1002200002360E2A02BE7DEF00F002360E2A02BE12
:100230007DEF00F002360E2A7DEF00F0010E0C6E0D
:10024000FBDE30EF01F0020E0C6E16DF30EF01F036
:10025000040E0C6E05DF30EF01F0080E0C6EF9DEB7
:10026000120073B409D01F0E7114016E0150000A00
:1002700003E1010E006E01D0006A1200F250026E1E
:10028000F29E0500FF6A0150FE6E0050FD6E02BE38
:10029000F28E1200220E0C6E086A096A0A6A0B6A54
:1002A0000C06D8B41FD0D8900B320A32093208326B
:1002B0000332023201320032D8A0F2D70C06D8B491
:1002C00009D0045008260550092206500A2207507A
:1002D0000B22EAD7045008260550092206500A22AC
:1002E00007500B2212000050086E0150006E0250A1
:1002F000016E0350026E036A0B6A0C6A9E0E036E57
:100300000A6A02AE90EF01F0081E001E011E021ED6
:10031000082AD8B4002AD8B4012AD8B4022A0A8EEE
:10032000020E0C6EADDE12000401C451390806E362
:10033000300EC45D03E3010E006E01D0006A1200AE
:1003400026C0C6F427C0C7F428C0C8F429C0C9F421
:100350000401C46BC56BC551120802E1C4518E087B
:1003600008E37FDF005201E004D00401C44BC52B39
:10037000F2D70401120EC55D02E18F0EC45D03E3E6
:100380007B0E006E24D0718071A020D026502710E3
:10039000281029101AE0C651C711C811C9110EE161
:1003A00032C3E1FF33C3E2FF050EE66E30C300F057
:1003B00031C301F063DF010E006E09D0010E0401AC
:1003C000C65F000EC75BC85BC95BDED7006A120060
:1003D000550EA76EAA0EA76E0E01BF811200550E14
:1003E000A76EAA0EA76E0E01BF911200A49EC4C4F0
:1003F00075FF26C0C5F427C0C6F428C0C7F429C0BD
:10040000C8F473A421D026502710281029101BE00F
:100410000401C551C611C711C8110EE132C3E1FF75
:1004200033C3E2FF040EE66E30C300F031C301F0C7
:1004300025DF010E006E3AD0010E0401C55F000EEB
:10044000C65BC75BC85BDDD726C0C5F427C0C6F452
:1004500028C0C7F429C0C8F4A4BE21D02650271054
:10046000281029101BE00401C551C611C711C8117D
:100470000EE132C3E1FF33C3E2FF040EE66E30C388
:1004800000F031C301F0FADE010E006E0FD0010E54
:100490000401C55F000EC65BC75BC85BDDD771BCDE
:1004A00002D0006A03D07184020E006E12000401B3
:1004B000C451200A09E0C4510D0804E3090EC45DCB
:1004C00001E302D0006A02D0010E006E1200C7B430
:1004D00009D01F0EC514016E0150000A03E1010E80
:1004E000006E01D0006A12007184120003500718D8
:1004F000D8A48AEF02F002500618D8A48AEF02F0BE
:1005000001500518D8A48AEF02F000500418D8B49E
:10051000D8841200D894120012000B800BAE99EF11
:1005200002F0026A0AAEFF0E026E016E006E0A361B
:100530000232FF0E1200025006180E6E086A096A97
:100540000B6A035007648EEF03F006500A6E068EA6
:10055000028E03500B6E0750036E000E0B64DEEF2D
:1005600002F00B50075ED8B47FEF03F0070E07646C
:100570004DEF03F0075E00C008F001C000F002C0BC
:1005800001F0026A074E7FEF03F0076422EF03F0E9
:10059000075E00C008F001C000F0016A074E7FEF5F
:1005A00003F0076400EF03F0075E00C008F0006A84
:1005B000074E7FEF03F00764E7EF02F00AC002F096
:1005C00005C001F004C000F0086AABEF04F0030EB0
:1005D0000764F2EF02F0075E08380F0B086E074E53
:1005E0007FEF03F0D8900832074E7FEF03F0D890EA
:1005F0000832074E7FEF03F0D89008327FEF03F008
:10060000030E076411EF03F0075E08380F0B086E46
:100610000038F00B082600380F0B006E074E7FEFF6
:1006200003F0D89000320832074E7FEF03F0D890E5
:1006300000320832074E7FEF03F0D89000320832C4
:100640007FEF03F0030E076439EF03F0075E08380D
:100650000F0B086E0038F00B082600380F0B006EE9
:100660000138F00B002601380F0B016E074E7FEFAB
:1006700003F0D890013200320832074E7FEF03F0CA
:10068000D890013200320832074E7FEF03F0D89045
:100690000132003208327FEF03F0030E07646AEF85
:1006A00003F0075E08380F0B086E0038F00B0826C1
:1006B00000380F0B006E0138F00B002601380F0BCD
:1006C000016E0238F00B012602380F0B026E074E46
:1006D0007FEF03F0D8900232013200320832074E29
:1006E0007FEF03F0D8900232013200320832074E19
:1006F0007FEF03F0D8900232013200320832096AEB
:10070000000E0EAE73EF04F0081E001E011E021E46
:10071000082A00220122022273EF04F00750D8A415
:1007200094EF03F0ABEF04F0096A02C00AF0028E06
:10073000068E0750035C076ED8B466EF04F0070E10
:10074000076434EF04F0075E0450096E0550046E30
:100750000650056E066A074E66EF04F0070E076442
:1007600009EF04F0075E0450096E0550046E056A37
:10077000074E66EF04F0070E0764E7EF03F0075E2D
:100780000450096E046A074E66EF04F0070E076412
:10079000CEEF03F00AC002F0ABEF04F0030E0764E3
:1007A000D9EF03F0075E09380F0B096E074E66EFAD
:1007B00004F0D8900932074E66EF04F0D890093261
:1007C000074E66EF04F0D890093266EF04F0030E8E
:1007D0000764F8EF03F0075E09380F0B096E043861
:1007E000F00B092604380F0B046E074E66EF04F079
:1007F000D89004320932074E66EF04F0D8900432E4
:100800000932074E66EF04F0D8900432093266EFE1
:1008100004F0030E076420EF04F0075E09380F0BA5
:10082000096E0438F00B092604380F0B046E0538E6
:10083000F00B042605380F0B056E074E66EF04F02B
:10084000D890053204320932074E66EF04F0D89092
:10085000053204320932074E66EF04F0D8900532B3
:100860000432093266EF04F0030E076451EF04F01E
:10087000075E09380F0B096E0438F00B092604389F
:100880000F0B046E0538F00B042605380F0B056EB0
:100890000638F00B052606380F0B066E074E66EF7E
:1008A00004F0D8900632053204320932074E66EF62
:1008B00004F0D8900632053204320932074E66EF52
:1008C00004F0D8900632053204320932086A000E6C
:1008D0000EAE73EF04F0091E041E051E061E092A43
:1008E0000422052206220950082604500022055041
:1008F0000122065002220EBE8AEF04F0D8A099EF22
:1009000004F00232013200320832033E99EF04F063
:10091000A5EF04F0D8B09FEF04F0000E081E001EF3
:10092000011E021E082A0022012202220A7E9FEFD7
:1009300004F0010E0C6E40EC00F0ADEF04F0020E7E
:100940000C6E40EC00F0ADEF04F0040E0C6E30ECD9
:1009500000F0ADEF04F0000E0C6E12000C6A0E6A8F
:100960000250D8A4C7EF04F001C002F000C001F0AB
:10097000006A0E860250D8A4C7EF04F001C002F04E
:10098000016A0E960E880250D8B4D9EF04F00E50CA
:10099000035ED8A4D8A0DFEF04F0D89002BEE5EF44
:1009A00004F0003601360236032ECEEF04F0DFEFFE
:1009B00004F0010E0C6E29EC00F0E9EF04F0020ED9
:1009C0000C6E1CEC00F0E9EF04F0040E0C6E3CEC35
:1009D00000F012000B6A0B86FF0E12000A6A035029
:1009E000D8A40A800750D8A40A820A50D8B451EF7C
:1009F00005F0030AD8B40AEF05F00AB005EF05F0D8
:100A000006AE4FEF05F04DEF05F002AE4DEF05F0ED
:100A10004FEF05F00250800B0A6E029E0650800BCD
:100A2000069E0A18D8B41BEF05F00A50D8B44DEF53
:100A300005F04FEF05F00750035CD8B425EF05F043
:100A4000D8A041EF05F047EF05F00650025CD8B49E
:100A50002FEF05F0D8A041EF05F047EF05F0055066
:100A6000015CD8B439EF05F0D8A041EF05F047EFAD
:100A700005F00450005CD8B451EF05F0D8B047EF52
:100A800005F00A52D8B44FEF05F04DEF05F00A52C9
:100A9000D8B44DEF05F04FEF05F0D8801200D89094
:100AA0001200D880D88412001200086A096A000E69
:100AB00007620364DAEF05F0025006180A6E075069
:100AC00003267E0ED8A06BEF05F0035ED8B0DFEFF3
:100AD00005F06FEF05F0035ED8A0E4EF05F0028E9D
:100AE000068E02C00EF001C00BF000C00DF00050E9
:100AF0000402F4CF0CF001500502F4CF00F0F3CF64
:100B000008F00402F3500C26F4500822000E0022D4
:100B10000D500502F3500C26F4500822000E00225E
:100B200002500402F3500826F4500022025005023D
:100B3000016A000E0122F3500026F45001220D50EC
:100B40000602F3500826F4500022026A000E012229
:100B500002220B500602F3500026F4500122000E30
:100B600002220E500602F3500126F450022202BE69
:100B7000C2EF05F008360036013602360306D8B457
:100B8000E4EF05F0D5EF05F0D880800E0864003062
:100B9000000E002201220222D8A0D5EF05F0023279
:100BA00001320032034ADFEF05F00AAE029E000E6A
:100BB000E7EF05F0010E29EC00F0E7EF05F0020E7B
:100BC00030EC00F0E7EF05F0040E1CEC00F0120032
:100BD000A0EC01F0780E0401C46F08DC31EC01F0E8
:100BE0000050000A01E1FAD7400E0401C46FF6EC90
:100BF00001F031EC01F00050000A01E1FAD7B9C46C
:100C0000C4F4F6EC01F063DC0050000A01E1FBD70C
:100C10006BDC120000C008F00150006E016A026A2D
:100C2000036A0B6A0C6A016A026A036A960E036E13
:100C30000A6A00AE22EF06F0081E001E082AD8B489
:100C4000002A0A8E00C001F008C000F0086A026A9B
:100C500085DE1200A0EC01F0780E0401C46FF6EC02
:100C600001F031EC01F00050000A01E1FAD7800EEA
:100C70000401C46FF6EC01F031EC01F00050000A01
:100C800001E1FAD7B9C4C4F4F6EC01F031EC01F09B
:100C90000050000A01E1FAD727DC31EC01F00050E6
:100CA000000A01E1FAD71200086A096A100E0C6EF8
:100CB0000134083609360450085E0550D8A0053CBA
:100CC000095ED8B007D0045008260550D8B0053CBE
:100CD0000926D890003601360C2EEAD71200086A91
:100CE000080E0C6E003408360450085ED8B002D0EE
:100CF0000826D89000360C2EF5D712000B6A035048
:100D0000D8B4C4EF06F002500A6E028E8E0E035E57
:100D100003AEC8EF06F0036C080E035CD8A0A3EF87
:100D200006F0036E013602C001F0026A080E035C91
:100D3000D8A0A3EF06F0036E0136016A0350D8A4D1
:100D4000D890ADEF06F00350D8B4ADEF06F0D890D0
:100D500002320132032EA7EF06F00BBC01A0BAEF5E
:100D600006F0D8A0BAEF06F0012AD8B4022A02BED3
:100D7000D7EF06F00AAEDDEF06F0021E011E012AD3
:100D8000D8B4022ADDEF06F0026A016ADDEF06F050
:100D90000B800BAEE1EF06F0026A0AAEE1EF06F05F
:100DA000FF0E026E016E0A360232E1EF06F0010E0E
:100DB0000C6E8DEC02F0E3EF06F0000E0C6EE3EF2C
:100DC00006F0FF0E0C6E0150006E0250016E120014
:100DD0000B6A0C6A086A0350D8B46CEF07F002C0C3
:100DE0000AF0028E9E0E035E03AE5CEF07F0036C0A
:100DF000080E035CD8A029EF07F0036E083600C088
:100E000008F001C000F002C001F0026A080E035CA5
:100E1000D8A029EF07F0036E083600C008F001C023
:100E200000F0016A080E035CD8A029EF07F0036EFA
:100E3000083600C008F0006A080E035CD8A029EF4D
:100E400007F0036E0836086A0350D8A4D89035EF2F
:100E500007F00350D8B435EF07F0D89002320132D2
:100E600000320832032E2DEF07F00BBC08A046EF2E
:100E700007F0D8A046EF07F0082AD8B4002AD8B463
:100E8000012AD8B4022A02BE70EF07F00AAE6CEF56
:100E900007F0021E011E001E081E082AD8B4002AF0
:100EA000D8B4012AD8B4022A6CEF07F0026A016AAA
:100EB000006A086A6CEF07F00B800BAE77EF07F063
:100EC000026A0AAE77EF07F0026E016E006E086EDE
:100ED0000A36023277EF07F00C6A000E78EF07F05F
:100EE000010E0C6E000E8DEC02F078EF07F0FF0E95
:100EF0000250036E0150026E0050016E0850006EE9
:100F00001200067E9BEC02F012000401B951180891
:100F100008E3B9510D0804E2110EB95D01E201D0F8
:100F200002D0006AFAD1BA51000AD8A48FD0BC53BB
:100F300002E0EFEC01F042D0BBC4C0FE82D0BBC4E3
:100F4000C1FE7FD0BBC4C2FE7CD0BBC4C3FE79D07F
:100F5000BBC4C4FE76D0BBC4C5FE73D0BBC4C6FE42
:100F600070D0BBC4C7FE6DD0BBC4C8FE6AD0BBC4C2
:100F7000C9FE67D0BBC4CAFE64D0BBC4CBFE61D07F
:100F8000BBC4CCFE5ED0BBC4CDFE5BD0BBC4D1FE27
:100F900058D0BBC4D2FE55D0BBC4D3FE52D0BBC4C4
:100FA000D4FE4FD0BBC4D5FE4CD0BBC4D6FE49D076
:100FB000BBC4D7FE46D0BBC4D8FE43D00401B95150
:100FC000000ABAE0B951010ABAE0B951020ABAE01E
:100FD000B951030ABAE0B951040ABAE0B951050A95
:100FE000BAE0B951060ABAE0B951070ABAE0B951F4
:100FF000080ABAE0B951090ABAE0B9510A0ABAE0D6
:10100000B9510B0ABAE0B9510C0ABAE0B9510D0A4C
:10101000BAE0B951110ABAE0B951120ABAE0B951AD
:10102000130ABAE0B951140ABAE0B951150ABAE084
:10103000B951160ABAE0B951170ABAE0B951180AFB
:10104000BAE00401BC5302E0E8EC01F00401BA513B
:10105000010AD8A477D0BC5302E0EFEC01F036D0FF
:10106000B9C4E1FE6AD0B9C4E2FE67D0B9C4E3FEF8
:1010700064D0B9C4E4FE61D0B9C4E6FE5ED0B9C4A0
:10108000E7FE5BD0B9C4E8FE58D0B9C4E9FE55D03C
:10109000B9C4EAFE52D0B9C4F2FE4FD0B9C4F3FECF
:1010A0004CD0B9C4F4FE49D0B9C4F7FE46D0B9C497
:1010B000F8FE43D0B9C4FCFE40D0B9C4FDFE3DD01B
:1010C000B9C4FEFE3AD0B9C4FFFE37D00401BB510B
:1010D000000AC6E0BB51010AC6E0BB51020AC6E0E5
:1010E000BB51030AC6E0BB51040AC6E0BB51050A66
:1010F000C6E0BB51060AC6E0BB51070AC6E0BB51B9
:10110000080AC6E0BB51090AC6E0BB510A0AC6E09C
:10111000BB510B0AC6E0BB510C0AC6E0BB510D0A1D
:10112000C6E0BB510E0AC6E0BB510F0AC6E0BB5178
:10113000100AC6E0BB51110AC6E00401BC5302E02C
:10114000E8EC01F09AD00401BAB102D0929001D03B
:101150009280E1D00401BAB102D0929201D0928281
:10116000DAD00401BAB102D0929A01D0928AD3D0D7
:101170000401BAB102D0939001D09380CCD0040185
:10118000BAB102D0939201D09382C5D00401BAB112
:1011900002D0939401D09384BED00401BAB102D09E
:1011A000939601D09386B7D00401BAB102D0939838
:1011B00001D09388B0D00401BAB102D0939A01D083
:1011C000938AA9D00401BAB102D0939C01D0938C28
:1011D000A2D00401BAB102D0939E01D0938E9BD0CD
:1011E0000401BAB102D0949001D0948094D004014B
:1011F000BAB102D0949201D094828DD00401BAB1D8
:1012000002D0949401D0948486D00401BAB102D063
:10121000949C01D0948C7FD00401BAB102D0949EEA
:1012200001D0948E78D00401BAB102D0959401D047
:10123000958471D00401BAB102D0959601D09586FB
:101240006AD00401BAB102D0959801D0958863D0D4
:101250000401BAB102D0959A01D0958A5CD00401FC
:10126000BAB102D0959C01D0958C55D00401BAB189
:1012700002D0959E01D0958E4ED00401B951000A3E
:10128000D8B461D7B951010AD8B464D7B951020AA8
:10129000D8B467D7B951030AD8B46AD7B951040A88
:1012A000D8B46DD7B951050AD8B470D7B951060A68
:1012B000D8B473D7B951070AD8B476D7B951080A48
:1012C000D8B479D7B951090AD8B47CD7B9510A0A28
:1012D000D8B47FD7B9510B0A83E0B9510C0A87E023
:1012E000B9510D0A8BE0B951110A8FE0B951120AB8
:1012F00093E0B951130A97E0B951140A9BE0B95130
:10130000150A9FE0B951160AA3E0B951170AA7E0E0
:10131000B951180AABE0FF0E006E12000401BB5178
:10132000BC1108E0BBC4E1FFBCC4E2FFB9C4E6FFE6
:10133000BAC4E6FFB9C4E9FFBAC4EAFFEECF00F0D1
:1013400000C0BFF400C0C4F457EC02F0005203E048
:10135000B94BBA2BEFD7BD6B000EBFBFFF0E006EAF
:10136000000E001802E12D0EBF1905E1010EBD6F40
:10137000B94BBA2B0CD0000EBFBFFF0E006E000E93
:10138000001802E12B0EBF1902E1B94BBA2BBF6B5B
:10139000C06BC16BC26BC36BBE6BBDB90BD0B9C4A4
:1013A000E9FFBAC4EAFFEE502E0A04E1BD89B94B49
:1013B000BA2B59D0B9C4E9FFBAC4EAFFEECFC4F4DE
:1013C00094EC01F0005201E14FD0BD83000EBFBF8D
:1013D000FF0E000A02E1080EBF1940E0BDA901D0CE
:1013E000BE07BF2BC0C400F0C1C401F0C2C402F0EC
:1013F000C3C403F00A0E046E000E056E066E076E7F
:101400004AEC01F000C0C0F401C0C1F402C0C2F453
:1014100003C0C3F400000000B9C4E9FFBAC4EAFF86
:10142000300EEE5C006E016A000E015A000E01BE25
:10143000FF0E026E036EC0510026C1510122C2513F
:101440000222C351032200C0C0F401C0C1F402C093
:10145000C2F403C0C3F40000000003D0BDB901D042
:10146000BE2BB94BBA2B99D7BF6BB9C4E9FFBAC42D
:10147000EAFFEE50650A08E0B9C4E9FFBAC4EAFF22
:10148000EE50450A01E068D0B94BBA2BB9C4E9FF68
:10149000BAC4EAFFEE502D0A04E1BD87B94BBA2B5E
:1014A00009D0B9C4E9FFBAC4EAFFEE502B0A02E141
:1014B000B94BBA2BB9C4E9FFBAC4EAFFEE50300AFF
:1014C00003E1B94BBA2BF6D7B9C4E9FFBAC4EAFFB6
:1014D000EECFC4F494EC01F0005239E0B9C4E9FF56
:1014E000BAC4EAFF300EEE5CBF6FB94BBA2BB9C479
:1014F000E9FFBAC4EAFFEECFC4F494EC01F0005265
:1015000026E00A0EBF03F3CFBFF4B9C4E9FFBAC4A3
:10151000EAFF300EEE5C006E0050BF27B94BBA2BCD
:10152000B9C4E9FFBAC4EAFFEECFC4F494EC01F009
:1015300000520DE00A0EBF03F3CFBFF4B9C4E9FFB8
:10154000BAC4EAFF300EEE5C006E0050BF27BDA7A4
:1015500003D0BF510008BF6FBF51BE27000EBC199A
:1015600002E1000EBB190AE0BDA308D0BBC4E1FF35
:10157000BCC4E2FFB9C4E6FFBAC4E6FFC0C400F0D1
:10158000C1C401F0C2C402F0C3C403F073EC01F0A3
:1015900000C0C0F401C0C1F402C0C2F403C0C3F46F
:1015A000046A056A066A076AC0C400F0C1C401F093
:1015B000C2C402F0C3C403F076EC02F0010ED8A45A
:1015C000000E006E005205E0006A016A026A036ABA
:1015D00004D1800EBE19006E800E000A005CD8B0E7
:1015E00073D0BE510008BE6F800EBE19006E800E13
:1015F0000A0A005C1DE3C0C400F0C1C401F0C2C40B
:1016000002F0C3C403F0FF0E046EE60E056E5B0E1F
:10161000066E5D0E076E55EC05F000C0C0F401C00B
:10162000C1F402C0C2F403C0C3F40A0EBE5FDCD72B
:10163000BE51000A1CE0C0C400F0C1C401F0C2C425
:1016400002F0C3C403F0CD0E046ECC0E056E4C0E3A
:10165000066E7B0E076E55EC05F000C0C0F401C0AD
:10166000C1F402C0C2F403C0C3F4BE07E1D7010E47
:10167000046E000E056E000E066E010E076EC0C4ED
:1016800000F0C1C401F0C2C402F0C3C403F0EEEC28
:1016900004F0010ED8B0000E006E005214E0BDA19F
:1016A00009D0010E006E000E016E800E026E030E58
:1016B000036E93D0010E006E000E016E000E026EDE
:1016C000010E036E8AD072D0800E000A006E800E6A
:1016D000BE19005C6BE20A0EBE5D1DE3C0C400F0E3
:1016E000C1C401F0C2C402F0C3C403F0F90E046E19
:1016F000020E056E150E066EA00E076E55EC05F077
:1017000000C0C0F401C0C1F402C0C2F403C0C3F4FD
:101710000A0EBE5FE0D7BE51000A1CE0C0C400F054
:10172000C1C401F0C2C402F0C3C403F0000E046ED1
:10173000000E056E200E066E820E076E55EC05F04B
:1017400000C0C0F401C0C1F402C0C2F403C0C3F4BD
:10175000BE07E1D7C0C404F0C1C405F0C2C406F09E
:10176000C3C407F0FF0E006EFF0E016E7F0E026E07
:10177000FF0E036EEEEC04F0010ED8B0000E006E0A
:10178000005214E0BDA109D0FF0E006EFF0E016EE5
:10179000FF0E026EFF0E036E20D0FF0E006EFF0ED6
:1017A000016E7F0E026EFF0E036E17D0BDA10DD02D
:1017B000000EC019006E000EC119016E800EC21914
:1017C000026E000EC319036E08D0C0C400F0C1C47D
:1017D00001F0C2C402F0C3C403F012000B6A0A6A2B
:1017E000096A00500402F4CF09F0F3CF08F0015069
:1017F0000502F4CF0BF0F3CF0AF000500502F350CE
:101800000926F4500A22E86A0B2201500402F35020
:101810000926F4500A22E86A0B2208C000F009C029
:1018200001F00AC002F00BC003F012000450000ADD
:1018300012E10550000A0FE10650000A0CE10750C2
:10184000000A09E1FF0E006EFF0E016E7F0E026EB0
:10185000FF0E036EA8D0086A096A0750D8B4C1EF1A
:101860000CF00350D8B4C6EF0CF0025006180A6E04
:10187000028E068E0E6A02C008F001C00CF000C095
:101880000DF004500D5E0550D8A0053C0C5E0650CE
:10189000D8A0063C085E086A0C6A0D6AD8A058EF0A
:1018A0000CF0D8900232013200320832010E0E6E76
:1018B0000750035ED8A065EF0CF07E0E0E240326C1
:1018C000D8B0CBEF0CF06BEF0CF07E0E0E2403269D
:1018D000D8A0D0EF0CF0180E0B6E0D360C36083673
:1018E0000036013602360E360450005E0550D8A090
:1018F000053C015E0650D8A0063C025E06340E127E
:101900000EA086EF0CF00D8091EF0CF00450002635
:101910000550D8B0053C01260650D8B0062802264E
:101920000D900B2E6DEF0CF0B7EF0CF0D890003649
:10193000013602360E360450005E0550D8A0053C34
:10194000015E0650D8A0063C025E06340E10010B64
:101950000D26D8B00C2AD8B4082AD8A4B7EF0CF0BA
:1019600008320C320D32032AD8B4CBEF0CF00AAE99
:10197000089E0850026E0C50016E0D50006ED3EFA1
:101980000CF0010EEAEC04F0D3EF0CF0020E29EC9F
:1019900000F0D3EF0CF0040E30EC00F0D3EF0CF0BD
:1019A000080E1CEC00F012000401A851000805E329
:1019B000070EA96F000EAA6F12D0A851160805E2F3
:1019C000170EAB6F000EAC6F06D0A851010FAB6FB6
:1019D000AC6B000EAC23ABC4A9F4ACC4AAF4A9C48C
:1019E000B3F4AAC4B4F4AD6BAE6B046A056A066ABC
:1019F000076AA2C400F0A3C401F0A4C402F0A5C405
:101A000003F0EEEC04F0010ED8B0000E006E0052B0
:101A100009E0A6C4E1FFA7C4E2FF2D0EE66EA64BC7
:101A2000A72BA47FA2C404F0A3C405F0A4C406F0AD
:101A3000A5C407F0006A016A026A036AEEEC04F0CA
:101A4000010ED8B0000E006E005237E0000E046E9A
:101A5000000E056E000E066E7F0E076EA2C400F02B
:101A6000A3C401F0A4C402F0A5C403F0EEEC04F09A
:101A7000010ED8B0000E006E00521FE0A2C400F0AC
:101A8000A3C401F0A4C402F0A5C403F0000E046EC8
:101A9000000E056E200E066E820E076E55EC05F0E8
:101AA00000C0A2F401C0A3F402C0A4F403C0A5F4D2
:101AB000010EAD5F000EAE5BC9D7000E046E000EC6
:101AC000056E200E066E820E076EA2C400F0A3C43F
:101AD00001F0A4C402F0A5C403F0EEEC04F0000E83
:101AE000D8B0010E006E00521DE0000E046E000E14
:101AF000056E200E066E820E076EA2C400F0A3C40F
:101B000001F0A4C402F0A5C403F090DE00C0A2F46A
:101B100001C0A3F402C0A4F403C0A5F40401AD4BBA
:101B2000AE2BCBD7AD51B327AE51B423010EAF6F5F
:101B3000000EB06F000EB56F000EB66F000EB76FDF
:101B40007F0EB86F800EB019006E800EB419005C65
:101B500002E1B351AF5D1DE2000E046E000E056E92
:101B6000200E066E820E076EB5C400F0B6C401F0FA
:101B7000B7C402F0B8C403F059DE00C0B5F401C028
:101B8000B6F402C0B7F403C0B8F40401AF4BB02BF5
:101B9000D9D7000E046E000E056E000E066E800E84
:101BA000076EB5C400F0B6C401F0B7C402F0B8C403
:101BB00003F03CDEA2C404F0A3C405F0A4C406F004
:101BC000A5C407F09BEC02F000C0A2F401C0A3F48E
:101BD00002C0A4F403C0A5F4000E046E000E056E4E
:101BE000200E066E820E076EEEEC04F0000ED8B0EA
:101BF000010E006E00520BE0000E0401A26F000EF9
:101C0000A36F000EA46F7F0EA56FAD4BAE2B04012A
:101C1000800EAE19006E800E005C02E1000EAD5D1C
:101C200038E2A6C4E1FFA7C4E2FF300EE66EA64B81
:101C3000A72BA6C4E1FFA7C4E2FF2E0EE66EA64BBB
:101C4000A72B800EB419006E800E005C02E1000E1E
:101C5000B35D04E2B351AD5FB451AE5BFF0EAF6F45
:101C6000FF0EB06F800EAE19006E800EB019005CD2
:101C700002E1AF51AD5D0DE2A6C4E1FFA7C4E2FFF2
:101C8000300EE66EA64BA72B010EAF5F000EB05BC9
:101C9000E9D7AF6BB06B800EB019006E800EB4192F
:101CA000005C02E1B351AF5D63E2A2C400F0A3C4E3
:101CB00001F0A4C402F0A5C403F07EEC06F000C05D
:101CC000B1F401C0B2F4300E0026A6C4E1FFA7C4EF
:101CD000E2FF00C0E6FFA64BA72BB051AE1902E110
:101CE000AD51AF1908E1A6C4E1FFA7C4E2FF2E0E73
:101CF000E66EA64BA72BB1C400F0B2C401F00AEC0B
:101D000006F000C0B5F401C0B6F402C0B7F403C0D9
:101D1000B8F400C004F001C005F002C006F003C032
:101D200007F0A2C400F0A3C401F0A4C402F0A5C44B
:101D300003F081EC07F000C0A2F401C0A3F402C0DC
:101D4000A4F403C0A5F4000E046E000E056E200E70
:101D5000066E820E076E55EC05F000C0A2F401C0BD
:101D6000A3F402C0A4F403C0A5F4AF4BB02B93D7E7
:101D7000A6C4E1FFA7C4E2FFE66A1200A2C402F013
:101D8000A3C403F002C000F003C001F0024A032A1A
:101D900000C0E9FF01C0EAFFEE5201E0F3D7040101
:101DA000A251025C006EA3510358016E010E005E49
:101DB000000E015A1200AFCF01F0ACA202D0AC98D5
:101DC000AC8801C000F01200840ED56E6D0ED76E87
:101DD000840ED66E01019293D08EF294F28A120094
:101DE0000401A66B050EA65D0AE2A651A425E16ECC
:101DF000000EA521E26E200EE66EA62BF3D7A651AB
:101E0000A425E16E000EA521E26EE66AA607A651A2
:101E1000A425A76F000EA521A86F0A0E046E000E60
:101E2000056EA2C400F0A3C401F054EC06F008C093
:101E300000F009C001F0300E0026A7C4E1FFA8C4DD
:101E4000E2FF00C0E6FF0A0E046E000E056EA2C49B
:101E500000F0A3C401F054EC06F000C0A2F401C0ED
:101E6000A3F4000E011802E1000E001801E102D0F7
:101E7000A607CDD71200A6C400F00401A6070052A1
:101E800028E0A2C4E9FFA3C4EAFFEE50000A0CE078
:101E9000A2C4E9FFA3C4EAFFA4C4D9FFA5C4DAFF22
:101EA000EE50DE1801E10FD0A2C4E9FFA3C4EAFF9F
:101EB000A4C4D9FFA5C4DAFFDE50EE5C006E016A4F
:101EC000000E015A08D00401A24BA32BA44BA52B52
:101ED000D2D7006A016A1200000E9EBA010E006E8F
:101EE0001200A2C4B9F4A3C4BAF40401BB6BBC6B66
:101EF0008EEC09F012000401A46BA56BA2C403F0E0
:101F0000A3C404F0A2C405F0A3C406F003C0E9FF13
:101F100004C0EAFFEE50200A04E1A451A51101E13A
:101F200010D0010EA46F000EA56F03C0E9FF04C01E
:101F3000EAFF05C0E1FF06C0E2FFEECFE6FF054A7B
:101F4000062A03C001F004C002F0034A042A01C0BB
:101F5000E9FF02C0EAFFEE50000AD8E1A2C400F097
:101F6000A3C401F01200A5C400F0016A026A036A6A
:101F7000FF0E0016000E011600C0AAF401C0ABF45B
:101F80007F0E005C026E000E0158036E02C0AAF4C0
:101F900003C0ABF4800E0318006E800E005C02E1FB
:101FA000000E025C22E2046A056A066A076AA2C49D
:101FB00000F0A3C401F0A4C402F0A5C403F0EEEC49
:101FC00004F0010ED8B0000E006E005209E0000EC1
:101FD000006E000E016E800E026E7F0E036E5CD0EE
:101FE000006A016A026A036A57D00401AB51000813
:101FF00002E1AA51180809E2A2C400F0A3C401F04A
:10200000A4C402F0A5C403F047D0A2C400F0A3C446
:1020100001F0A4C402F0A5C403F0E8EC06F073ECF0
:1020200001F000C0A6F401C0A7F402C0A8F403C0E8
:10203000A9F400C004F001C005F002C006F003C01E
:1020400007F0A2C400F0A3C401F0A4C402F0A5C428
:1020500003F0EEEC04F0010ED8B0000E006E00525A
:1020600013E0000E046E000E056E000E066E7F0E6D
:10207000076EA6C400F0A7C401F0A8C402F0A9C46A
:1020800003F081EC07F008D0A6C400F0A7C401F06B
:10209000A8C402F0A9C403F01200200E0401B96F15
:1020A0002AEC06F00401B96B2AEC06F0210E0401BB
:1020B000B96F2AEC06F0A2C4B9F42AEC06F00401C8
:1020C000A2510F0FB96F2AEC06F0220E0401B96F6E
:1020D0002AEC06F0010E0401B96F2AEC06F0030E9B
:1020E0000401B96F2AEC06F00401A46BA56B800E05
:1020F000A519006E800E005C02E1300EA45D2EE298
:10210000030E006E000E016EA3C404F0000E056EF7
:10211000EEEC0BF0400E0024E96E000E0120EA6E9A
:10212000E9CFE9FFEACFEAFFA451EE24F66EA5510C
:10213000EE20F76E000EA5BFFF0EEE20F86EF6CF74
:10214000F6FFF7CFF7FFF8CFF8FF0900F5CFB9F4A6
:10215000E8EC05F00401A44BA52BC9D7120004013B
:10216000A56B030EA55D0AE2A551A325E16E000E45
:10217000A421E26E200EE66EA52BF3D7A551A32570
:10218000E16E000EA421E26EE66AA507A551A32523
:10219000A66F000EA421A76F0A0E046EA2C400F061
:1021A0006FEC06F008C000F0300E0026A6C4E1FF78
:1021B000A7C4E2FF00C0E6FF0A0E046EA2C400F04E
:1021C0006FEC06F000C0A2F40050000A01E102D05A
:1021D000A507DCD71200030E0D6E0D2EFED70000F2
:1021E00000001200A2C404F0A3C405F004C0E9FF7B
:1021F00005C0EAFFEE5203E0044A052AF7D704C0FF
:1022000002F005C003F0044A052AA4C400F0A5C4E6
:1022100001F00401A44BA52B00C0E9FF01C0EAFFB7
:1022200002C0E1FF03C0E2FFEECFE6FF02C0E9FF1C
:1022300003C0EAFFEE5201E0E2D7A2C400F0A3C45B
:1022400001F012000401A351B00FB96F2AEC06F09F
:102250000F0E0401A215B96F2AEC06F0F00E04016E
:10226000A215B96FB933B99FB933B99FB933B99FC3
:10227000B933B99FB9892AEC06F012000D0E04019A
:10228000CA6F15EC00F00A0E0401CA6F15EC00F0DD
:102290001200C70E0D6E0D2EFED7000000001200BA
:1022A0000401A56BA2C4E9FFA3C4EAFFEECFA4F426
:1022B000A451000A0FE0A4C4CAF415EC00F0040114
:1022C000A52BA551A225E96E000EA321EA6EEECF43
:1022D000A4F4EED71200A2C4B9F4A3C4BAF4A4C4FF
:1022E000BBF40401BC6B85EC07F01200A2C404F03F
:1022F000A3C405F004C002F005C003F0044A052A97
:10230000A4C400F0A5C401F00401A44BA52B00C097
:10231000E9FF01C0EAFF02C0E1FF03C0E2FFEECF28
:10232000E6FF02C0E9FF03C0EAFFEE5201E0E2D798
:10233000A2C400F0A3C401F01200A2C4E9FFA3C428
:10234000EAFFEE500401A41905E1A2C400F0A3C401
:1023500001F010D0A2C400F0A3C401F0A24BA32B43
:1023600000C0E9FF01C0EAFFEECF00F00052E5E156
:10237000006A016A1200080E0C6EC10E0D6E0D2E61
:10238000FED70C2EFCD7000000001200A4C4F6FFFC
:10239000A5C4F7FFA6C4F8FF0900F5CF00F000526E
:1023A00018E0A4C4F6FFA5C4F7FFA6C4F8FF09000F
:1023B000F5CF00F0A2C4E1FFA3C4E2FF00C0E6FF36
:1023C0000401A24BA32B010EA427000EA523A623D4
:1023D000DDD7A2C4E1FFA3C4E2FFE66A1200A2C4F3
:1023E000F6FFA3C4F7FFA4C4F8FF0900F5CF00F07F
:1023F000005215E0ADB201D0FDD7A2C4F6FFA3C4D0
:10240000F7FFA4C4F8FF0900F5CFCAF40EEC00F002
:10241000010E0401A227000EA323A423E0D712007B
:102420000401A56BA2C4E9FFA3C4EAFFEECFA4F4A4
:10243000A451000A0FE0A4C4CAF40EEC00F0040199
:10244000A52BA551A225E96E000EA321EA6EEECFC1
:10245000A4F4EED712000D0E0401CA6F0EEC00F0CA
:102460000A0E0401CA6F0EEC00F01200020E0C6E90
:10247000350E0D6E0D2EFED70C2EFCD70000000081
:102480001200A2C4F6FFA3C4F7FFA4C4F8FF09001A
:10249000F5CF00F0005215E0A8B201D0FDD7A2C4DC
:1024A000F6FFA3C4F7FFA4C4F8FF0900F5CFCAF4F0
:1024B00015EC00F0010E0401A227000EA323A423B3
:1024C000E0D712000401966B976B010E9A6F170EFE
:1024D000A26F040EA36F52DC00C098F401C099F4FF
:1024E000070E946F000E956F800E9519006E800E8A
:1024F0009919005C02E19851945DD8B000D2D5D111
:10250000170E9425E96E040E9521EA6EE9CFE9FFD6
:10251000EACFEAFFEECF01F001502C0A10E1880E5D
:102520009625E16E040E9721E26EE1CFE1FFE2CF46
:10253000E2FFE66A966B976B020E9A6FDDD1880E0A
:102540009625E16E040E9721E26E170E9425E96E32
:10255000040E9521EA6EE9CFE9FFEACFEAFFEECF5C
:1025600000F0E1CFE1FFE2CFE2FF00C0E6FF964BD3
:10257000972BC2D1170E9425E96E040E9521EA6EB1
:10258000E9CFE9FFEACFEAFFEECF01F001502C0AD4
:1025900010E1780E9625E16E040E9721E26EE1CFF0
:1025A000E1FFE2CFE2FFE66A966B976B030E9A6F4C
:1025B000A3D1780E9625E16E040E9721E26E170ED8
:1025C0009425E96E040E9521EA6EE9CFE9FFEACF82
:1025D000EAFFEECF00F0E1CFE1FFE2CFE2FF00C083
:1025E000E6FF964B972B88D1170E9425E96E040EC3
:1025F0009521EA6EE9CFE9FFEACFEAFFEECF01F0DD
:1026000001502C0A05E1966B976B040E9A6F74D1FA
:10261000170E9425E96E040E9521EA6EE9CFE9FFC5
:10262000EACFEAFFEECF00F000C077F4964B972B8D
:1026300063D1170E9425E96E040E9521EA6EE9CF59
:10264000E9FFEACFEAFFEECF01F001502C0A10E1DA
:102650008E0E9625E16E030E9721E26EE1CFE1FF2B
:10266000E2CFE2FFE66A966B976B050E9A6F44D154
:102670008E0E9625E16E030E9721E26E170E9425BD
:10268000E96E040E9521EA6EE9CFE9FFEACFEAFF91
:10269000EECF00F0E1CFE1FFE2CFE2FF00C0E6FFC6
:1026A000964B972B29D1170E9425E96E040E952190
:1026B000EA6EE9CFE9FFEACFEAFFEECF01F0015081
:1026C0002C0A05E1966B976B060E9A6F15D1170EC3
:1026D0009425E96E040E9521EA6EE9CFE9FFEACF71
:1026E000EAFFEECF00F000C09EF3964B972B04D18B
:1026F000170E9425E96E040E9521EA6EE9CFE9FFE5
:10270000EACFEAFFEECF01F001502C0A05E1966B0B
:10271000976B070E9A6FF0D0170E9425E96E040E92
:102720009521EA6EE9CFE9FFEACFEAFFEECF00F0AC
:1027300000C089F3964B972BDFD0170E9425E96ED6
:10274000040E9521EA6EE9CFE9FFEACFEAFFEECF6A
:1027500001F001502C0A10E18A0E9625E16E030E5D
:102760009721E26EE1CFE1FFE2CFE2FFE66A966BEE
:10277000976B080E9A6FC0D08A0E9625E16E030EF5
:102780009721E26E170E9425E96E040E9521EA6EEC
:10279000E9CFE9FFEACFEAFFEECF00F0E1CFE1FFBA
:1027A000E2CFE2FF00C0E6FF964B972BA5D0170EB5
:1027B0009425E96E040E9521EA6EE9CFE9FFEACF90
:1027C000EAFFEECF01F001502C0A10E1FF0E962532
:1027D000E16E030E9721E26EE1CFE1FFE2CFE2FF6F
:1027E000E66A966B976B090E9A6F86D0FF0E962558
:1027F000E16E030E9721E26E170E9425E96E040E2A
:102800009521EA6EE9CFE9FFEACFEAFFEECF00F0CB
:10281000E1CFE1FFE2CFE2FF00C0E6FF964B972B4E
:102820006BD0170E9425E96E040E9521EA6EE9CF60
:10283000E9FFEACFEAFFEECF01F001502C0A10E1E8
:10284000070E9625E16E040E9721E26EE1CFE1FFBF
:10285000E2CFE2FFE66A966B976B0A0E9A6F4CD056
:10286000070E9625E16E040E9721E26E170E942551
:10287000E96E040E9521EA6EE9CFE9FFEACFEAFF9F
:10288000EECF00F0E1CFE1FFE2CFE2FF00C0E6FFD4
:10289000964B972B31D098C494F499C495F42CD0CE
:1028A00098C494F499C495F427D09A51010AD8B4E5
:1028B00027D69A51020AD8B45DD69A51030AD8B4E1
:1028C00093D69A51040AD8B4B4D69A51050AD8B40A
:1028D000EAD69A51060AD8B40BD79A51070AD8B447
:1028E0002CD79A51080AD8B462D79A51090A99E0AC
:1028F0009A510A0AD0E0D4D7944B952BF5D59AC4B7
:1029000000F012000301806B816B000E815D02E11B
:10291000FF0E805D16E2170E8025E16E020E81210A
:10292000E26EE1CFE1FFE2CFE2FFE66A010E802531
:10293000006E000E8121016E00C080F301C081F3A2
:10294000E4D7826B836B806B816B9EAA02D0AFCF82
:1029500021F3216B0101936B946B9D8A12001F5030
:10296000010A08E1D00E0401A26F650EA36F000EEC
:10297000A46F35DD8E0E0401A26F030EA36F71EC00
:102980000FF000C089F001C08AF002C08BF003C0D4
:102990008CF0000E046E000E056E480E066E850E5D
:1029A000076E16EC0CF000C054F301C055F302C0E2
:1029B00056F303C057F300C0A2F401C0A3F402C051
:1029C000A4F403C0A5F4B3EC0FF000C094F401C06C
:1029D00095F402C096F403C097F494C454F395C4DC
:1029E00055F396C456F397C457F3000E046E000EC9
:1029F000056E480E066E850E076E89C000F08AC00F
:102A000001F08BC002F08CC003F016EC0CF094C403
:102A100004F095C405F096C406F097C407F081EC65
:102A200007F000C058F301C059F302C05AF303C0C5
:102A30005BF3000E046E000E056E480E066E850EEA
:102A4000076E55EC05F0000E046E000E056E700E5C
:102A5000066E840E076E16EC0CF094C404F095C458
:102A600005F096C406F097C407F09BEC02F000C096
:102A700089F001C08AF002C08BF003C08CF0040121
:102A80007751530A1AE189C000F08AC001F08BC067
:102A900002F08CC003F0000E046E000E056E800E76
:102AA000066E7F0E076E55EC05F000C089F001C080
:102AB0008AF002C08BF003C08CF089C0A2F48AC0F7
:102AC000A3F48BC0A4F48CC0A5F49F0EA66F030ED4
:102AD000A76F060EA86FD4EC0CF08E0EA26F030E3B
:102AE000A36F9F0EA46F030EA56F00DC0301226B82
:102AF000236B000E235D02E11F0E225D0FE25C0ED0
:102B00002225E16E030E2321E26EE1CFE1FFE2CF49
:102B1000E2FF200EE66E224B232BEBD75C6B5C0EA4
:102B20000401A26F030EA36F9F0EA46F030EA56F87
:102B300076EC11F05C0EA26F030EA36F2A0EA46F49
:102B4000000EA56FF2EC10F01F50010A15E19F0E68
:102B5000A26F030EA36F64DC200ECA6F0EEC00F0B0
:102B600077C4CAF40EEC00F0960E0401A26F650E55
:102B7000A36F000EA46F33DC780E0401A26F040E65
:102B8000A36F71EC0FF000C050F301C051F302C00D
:102B900052F303C053F3000E046E000E056E480E90
:102BA000066E850E076E16EC0CF000C054F301C0E3
:102BB00055F302C056F303C057F300C0A2F401C09E
:102BC000A3F402C0A4F403C0A5F4B3EC0FF000C05A
:102BD00094F401C095F402C096F403C097F494C431
:102BE00054F395C455F396C456F397C457F3000EA7
:102BF000046E000E056E480E066E850E076E50C3FD
:102C000000F051C301F052C302F053C303F016ECBD
:102C10000CF094C404F095C405F096C406F097C473
:102C200007F081EC07F000C058F301C059F302C06F
:102C30005AF303C05BF3000E046E000E056E480EDF
:102C4000066E850E076E55EC05F0000E046E000E44
:102C5000056E700E066E840E076E16EC0CF094C4B2
:102C600004F095C405F096C406F097C407F09BECF9
:102C700002F000C050F301C051F302C052F303C090
:102C800053F303019E51570A1AE150C300F051C398
:102C900001F052C302F053C303F0000E046E000EA5
:102CA000056E800E066E7F0E076E55EC05F000C0B7
:102CB00050F301C051F302C052F303C053F350C3A9
:102CC000A2F451C3A3F452C3A4F453C3A5F49F0EBA
:102CD0000401A66F030EA76F060EA86FD4EC0CF0CC
:102CE000780EA26F040EA36F9F0EA46F030EA56F44
:102CF00076EC11F05C0EA26F030EA36F9F0EA46F13
:102D0000030EA56FF2EC10F05C0EA26F030EA36F22
:102D10002C0EA46F000EA56FF2EC10F01F50010AEC
:102D200017E19F0EA26F030EA36F10EC12F0200E9E
:102D3000CA6F0EEC00F09EC3CAF40EEC00F09F0EBA
:102D40000401A26F650EA36F000EA46FEFEC11F0EB
:102D5000070E0401A26F040EA36F71EC0FF000C008
:102D60007CF301C07DF302C07EF303C07FF300C09B
:102D7000A2F401C0A3F402C0A4F403C0A5F49F0E02
:102D8000A66F030EA76F010EA86FD4EC0CF0070E10
:102D9000A26F040EA36F9F0EA46F030EA56F76ECB7
:102DA00011F05C0EA26F030EA36F9F0EA46F030EB3
:102DB000A56FF2EC10F01F50010A06E19F0EA26F02
:102DC000030EA36F10EC12F0200E0301746F756BED
:102DD0007B6B1F50010A2DE1540E0401A26F650E9A
:102DE000A36F000EA46FEFEC11F08A0E0401A26F26
:102DF000030EA36F10EC12F0680EA26F650EA36FA6
:102E0000000EA46FEFEC11F0FF0E0401A26F030E91
:102E1000A36F10EC12F0F80EA26F650EA36F000EF8
:102E2000A46FEFEC11F089C3CAF40EEC00F02BECA8
:102E300012F01F50010A12E10E0E0401A26F660E7D
:102E4000A36F000EA46F41EC12F05C0E0401A26FA0
:102E5000030EA36F50EC11F03EEC11F0120096C47B
:102E600001F0010E006E015004E000360090FF0FEB
:102E7000FBD700C098F4001E94C4E9FF95C4EAFF94
:102E80000050EF16120EE9260050EF16BBEC11F0C1
:102E900004019851EF12120EE95E36EC12F09851CF
:102EA000EF14976F9751000A000ED8A4010E976F88
:102EB000BBEC11F097C400F012000401A26BA36BED
:102EC00022EC11F00401956B080E955D28E29551F6
:102ED000B00FB96F2AEC06F0C70E0D6E0D2EFED79F
:102EE000000000000401B96B2AEC06F0100E04018A
:102EF000B96F2AEC06F00401966B800E965D0DE228
:102F000094C4B9F4E8EC05F0C70E0D6E0D2EFED793
:102F1000000000000401962BF0D7952BD5D71200A6
:102F2000070E0B6E170E0C6E6A0E0D6E0D2EFED771
:102F30000C2EFCD70B2EFAD7000012000401946B64
:102F4000EFEC01F0160E0401A26F010EA36F0C0E40
:102F5000A46F6BEC11F00050FF0A02E10401942B06
:102F60000401170EA26FA36B060EA46F6BEC11F099
:102F70000050FF0A02E10401942B0401120EA26F1B
:102F8000010EA36F070EA46F6BEC11F00050FF0A47
:102F900002E10401942B0401110EA26FA36B060E33
:102FA000A46F6BEC11F00050FF0A02E10401942BB6
:102FB000E8EC01F09C0E0C6ED70E0D6E0D2EFED7B8
:102FC0000C2EFCD794C400F012000900F5CFE6FFE8
:102FD0000006FBE10106F9E11200FF0E0F01486F48
:102FE000948E949C93988A88846A8D6A969C070E26
:102FF000D26E41919586958492909292928412001D
:103000002A0E03014C6F000E4D6FCA0E4E6F040E58
:103010004F6FFF0E386FFF0E396F000E3A6F000EC4
:103020003B6FFF0E3C6FFF0E3D6F000E3E6F000EBC
:103030003F6FFF0E406FFF0E416F000E426F000E9C
:10304000436FA88A900E9C6EA4AA03D0AACF00F06A
:10305000FBD712003EEC11F0380E0401A26F5C0E9B
:10306000A36F000EA46F41EC12F01D0E0401A26FBD
:103070005D0EA36F000EA46F41EC12F0860E0401EA
:10308000A26F5C0EA36F000EA46F41EC12F0D20E83
:103090000401A26F5C0EA36F000EA46F41EC12F04E
:1030A000CE0E0401A26F5B0EA36F000EA46F41EC65
:1030B00012F07F0E0401A26F630EA36F000EA46FC7
:1030C00041EC12F0520E0401A26F620EA36F000ECB
:1030D000A46F41EC12F0760E0401A26F5E0EA36F96
:1030E000000EA46F41EC12F0AD0E0401A26F5D0E54
:1030F000A36F000EA46F41EC12F0E70E0401A26F63
:10310000600EA36F000EA46F41EC12F0360E0401A6
:10311000A26F5E0EA36F000EA46F41EC12F0130EAF
:103120000401A26F610EA36F000EA46F41EC12F0B8
:103130008C0E0401A26F620EA36F000EA46F41EC0F
:1031400012F06F0E0401A26F620EA36F000EA46F47
:1031500041EC12F0150E0401A26F620EA36F000E77
:10316000A46F41EC12F03EEC11F0120094C4E9FFA0
:1031700095C4EAFFEECF96F4000E0401976F000E9F
:10318000976F000E971902E1200E961907E0000EC6
:10319000971902E1090E961901E003D0944B952B83
:1031A000E5D7986B996B9A6B9B6B000E971902E1B0
:1031B0002D0E961905E19A4B9B2B944B952B08D01D
:1031C000000E971902E12B0E961902E1944B952BF4
:1031D00094C4E9FF95C4EAFFEECF96F4000E976F12
:1031E000000E976F96C4C4F494EC01F0005219E0FD
:1031F00098C400F099C401F00A0E046E000E056E2A
:10320000EEEC0BF0300E965D026E000E9759036ED9
:1032100002500024986F03500120996F944B952B16
:10322000D7D79A519B1108E098510008006E99C4B5
:1032300001F0000E015604D098C400F099C401F0CA
:1032400012001C0E03014C6F000E4D6FCA0E4E6F24
:10325000040E4F6FB60E386F1D0E396F000E3A6FA9
:10326000000E3B6FD80E3C6F1E0E3D6F000E3E6F82
:10327000000E3F6FFF0E406FFF0E416F000E426F5A
:10328000000E436FAD8A900EAC6E948E949C9EAAF5
:1032900003D0AFCF00F0FBD71200040E0C6EE40E8B
:1032A0000D6E0D2EFED70C2EFCD700001200210E45
:1032B0000401B96F2AEC06F00401B96B2AEC06F0A0
:1032C0007F0E0401B96F2AEC06F0220E0401B96FDB
:1032D0002AEC06F00401B96B2AEC06F0070E040193
:1032E000B96F2AEC06F0D30E0401B96F2AEC06F090
:1032F000400E0401B96F2AEC06F00401A26BA36B27
:1033000022EC11F00401946B080E945D28E29451B4
:10331000B00FB96F2AEC06F0010E0401B96F2AEC68
:1033200006F0100E0401B96F2AEC06F0270E0D6EA0
:103330000D2EFED7000000000401956B800E955DF8
:103340000CE2B96BE8EC05F04F0E0D6E0D2EFED7BA
:10335000000000000401952BF1D7942BD5D72E0E39
:10336000B96F2AEC06F00401A26BA36B22EC11F0FA
:103370001200AE0E0401B96F2AEC06F00D0E0B6EB2
:103380002D0E0C6ED70E0D6E0D2EFED70C2EFCD70B
:103390000B2EFAD700000000AF0E0401B96F2AEC23
:1033A00006F0070E0B6E170E0C6E6A0E0D6E0D2ECC
:1033B000FED70C2EFCD70B2EFAD70000B00E04015E
:1033C000B96F2AEC06F00401B96B2AEC06F0070E7F
:1033D0000401B96F2AEC06F0200E0401B96F2AEC43
:1033E00006F0020E0401B96F2AEC06F0210E04016A
:1033F000B96F2AEC06F00401B96B2AEC06F07F0ED7
:103400000401B96F2AEC06F0220E0401B96F2AEC10
:1034100006F00401B96B2AEC06F0070E0401B96F3F
:103420002AEC06F0A10E0401B96F2AEC06F0A40EF6
:103430000401B96F2AEC06F0A60E0401B96F2AEC5C
:1034400006F0C80E0401B96F2AEC06F0D30E040191
:10345000B96F2AEC06F0400E0401B96F2AEC06F0B1
:10346000D50E0401B96F2AEC06F0800E0401B96F85
:103470002AEC06F0A80E0401B96F2AEC06F03F0E04
:103480000401B96F2AEC06F0D60E0401B96F2AECDC
:1034900006F0800E0401B96F2AEC06F0D90E040183
:1034A000B96F2AEC06F01F0E0401B96F2AEC06F082
:1034B000DA0E0401B96F2AEC06F00401B96B2AECAC
:1034C00006F0EE0E0401B96F2AEC06F0810E04013D
:1034D000B96F2AEC06F07F0E0401B96F2AEC06F0F2
:1034E0002E0E0401B96F2AEC06F0DB0E0401B96F51
:1034F0002AEC06F0400E0401B96F2AEC06F08D0E9E
:103500000401B96F2AEC06F0140E0401B96F2AEC1D
:1035100006F0AF0E0401B96F2AEC06F012008D0E12
:103520000401B96F2AEC06F0140E0401B96F2AECFD
:1035300006F0AF0E0401B96F2AEC06F012003D0E42
:103540000B6EE10E0C6E3F0E0D6E0D2EFED70C2E87
:10355000FCD70B2EFAD700000000120004019D6B6F
:103560009E6B9F6BA06BA16B94C4A0F495C4A1F457
:1035700094C4A2F495C4A3F422EC11F05FD1040129
:103580009F519625E96E000E9721EA6EE9CFE9FF7B
:10359000EACFEAFFEE50000A50E0050EA15D4DE2D1
:1035A0009F519625E96E000E9721EA6EE9CFE9FF5B
:1035B000EACFEAFF200EEE5C9D6FA051780809E289
:1035C00094C4A0F4A12B94C4A2F4A1C4A3F422EC4B
:1035D00011F004019E6B060E9E5D2BE2060E006E3E
:1035E000000E016E026E036E9DC404F0000E056EA7
:1035F000066E076E4AEC01F0A60E0026590E012257
:10360000000E02229E510024F66E000E0120F76E7D
:10361000000E0220F86EF6CFF6FFF7CFF7FFF8CFD7
:10362000F8FF0900F5CFB9F4E8EC05F004019E2B92
:10363000D2D7060EA0279F2BA2D70DD196C4A2F4F5
:1036400097C4A3F4BEEC0EF000C099F401C09AF444
:103650009F6B9F519625E96E000E9721EA6EE9CF88
:10366000E9FFEACFEAFFEE50000AD8B486D00F0E89
:103670009F5DD8B082D09F519625E96E000E9721AC
:10368000EA6EE9CFE9FFEACFEAFF200EEE5C9D6F1C
:10369000A0C4A2F4A1C4A3F422EC11F004019E6B17
:1036A000080E9E5D2BE2040E026E9DC400F0000E1B
:1036B000016E025005E0003600900136FF0FFAD788
:1036C0009E510026000E0122B60E0024F66E530E07
:1036D0000120F76E000EF86E000E01BEFF0EF822FC
:1036E000F6CFF6FFF7CFF7FFF8CFF8FF0900F5CFD9
:1036F000B9F4E8EC05F004019E2BD2D7A0C4A2F4E3
:10370000A151010FA36F22EC11F004019E6B080E72
:103710009E5D2FE2040E026E9DC400F0000E016E4D
:10372000025005E0003600900136FF0FFAD79E5197
:103730000026000E0122080E0026000E0122B60E01
:103740000024F66E530E0120F76E000EF86E000E88
:1037500001BEFF0EF822F6CFF6FFF7CFF7FFF8CF46
:10376000F8FF0900F5CFB9F4E8EC05F004019E2B51
:10377000CED7080EA0279F2B6CD76DD096C4A2F48D
:1037800097C4A3F4BEEC0EF000C09BF401C09CF4FF
:10379000800E026E800E0118025C02E100500008EB
:1037A0004BE29E6B800E006E800E9C19005C02E165
:1037B0009B519E5D41E2070E9E25996F9A6B000E0C
:1037C0009A239B51995F9C519A5B040E006E0050A6
:1037D00005E0993799919A37FF0FFAD79E519625B0
:1037E000E96E000E9721EA6EE9CFE9FFEACFEAFF22
:1037F000EECF01F001C09DF401502F080BE23A0E0C
:103800009D5D08E299C4A2F4300E9D5DA36F4DEC5E
:1038100010F010D09D512E0A07E199C4A2F40A0EAF
:10382000A36F4DEC10F006D099C4A2F4200EA36F44
:103830004DEC10F09E2BB6D70ED00DD00401985150
:10384000010AD8B49CD69851020AD8B4F7D6985138
:10385000030A94E0F2D71200200E0401B96F2AEC9B
:1038600006F00401B96B2AEC06F0210E0401B96FD1
:103870002AEC06F094C4B9F42AEC06F00401945141
:10388000070FB96F2AEC06F0220E0401B96F2AEC7B
:1038900006F095C4B9F42AEC06F004019551010F25
:1038A000B96F2AEC06F00401976B986B800E98199B
:1038B000006E800E005C02E1070E975D2EE2030EA3
:1038C000006E000E016E96C404F0000E056EEEEC64
:1038D0000BF0340E0024E96E000E0120EA6EE9CFF1
:1038E000E9FFEACFEAFF9751EE24F66E9851EE20F9
:1038F000F76E000E98BFFF0EEE20F86EF6CFF6FFC3
:10390000F7CFF7FFF8CFF8FF0900F5CFB9F4E8ECEF
:1039100005F00401974B982BC9D71200DBEC0EF091
:1039200094C424F095C425F0E4EC0EF08D0E04014F
:10393000A26F610EA36F000EA46F41EC12F094C44D
:10394000A2F495C4A3F4960E0401A46F040EA56F0F
:10395000F0EC0EF0960EA26F040EA36F50EC11F077
:10396000240EA26F650EA36F000EA46F41EC12F03F
:103970006CEC0FF00050000A04E1010192B301D099
:10398000F7D7DBEC0EF0120094C404F095C405F0F8
:1039900004019851991124E0010E985F000E995B83
:1039A00004C002F005C003F0044A052A96C400F0E2
:1039B00097C401F0964B972B00C0E9FF01C0EAFFC6
:1039C00002C0E1FF03C0E2FFEECFE6FF02C0E9FF65
:1039D00003C0EAFFEECF00F0005201E101D0D8D7DA
:1039E00098C400F099C401F0010E985F000E995B35
:1039F0000050011008E004C0E1FF05C0E2FFE66AE4
:103A0000044A052AEDD794C400F095C401F01200D1
:103A100094C400F00032009E0032009E0032009EEE
:103A20000032009ED80E0024F66E640EF76E000E73
:103A3000F722000EF86E000EF8220900F5CF00F014
:103A400095C4E1FF96C4E2FF00C0E6FF010E040149
:103A50009525E16E000E9621E26E0F0E9415006E14
:103A6000D80E0024F66E640EF76E000EF722000EDC
:103A7000F86E000EF8220900F5CF00F000C0E6FF56
:103A8000020E9525E16E000E9621E26EE66A1200A6
:103A90000401996B95AF0BD0010E996F2D0E0301A8
:103AA0009F6F0401941F951F944B952B04D0996B25
:103AB000200E03019F6F94C400F095C401F0013201
:103AC0000032019E01320032019E01320032019E1D
:103AD00001320032019E00C096F40A0E046E6FECB3
:103AE00006F00A0E046E6FEC06F008C000F0300E0F
:103AF0000024016E01C0A0F30150300A03E103016C
:103B0000200EA06F03010A0E046E96C400F06FEC45
:103B100006F008C000F0300E0024A16F94C497F4A2
:103B200095C498F40F0E04019415006E95C401F02D
:103B3000000E011600C097F401C098F4710E046ED7
:103B4000020E056EEEEC0BF000C09AF401C09BF47F
:103B50009AC497F49BC498F42E0E0301A26FE80E4A
:103B6000046E030E056E9AC400F09BC401F054EC81
:103B700006F0300E0024A36F640E046E000E056E76
:103B80009AC400F09BC401F054EC06F00A0E046ED7
:103B9000000E056E54EC06F008C000F009C001F0FC
:103BA000300E0024A46FA56BA66BA76BA00E0401BA
:103BB000A26F030EA36F7BEC0FF09951010A14E181
:103BC00096C400F0000E016EE80E046E030E056E42
:103BD000EEEC0BF097510024306E98510120316EBD
:103BE000000E326E336E18D096C400F0000E016ED7
:103BF000E80E046E030E056EEEEC0BF097510026F6
:103C00009851012200500008306E01C031F0000EC2
:103C10003156000E326E336E99C400F0120096C415
:103C200001F0010E006E015004E000360090FF0F1D
:103C3000FBD700C09AF4001E00C099F494C4E9FFB9
:103C400095C4EAFF0050EF16120EE9260401986BA6
:103C50009851070816E398C400F097C401F000508B
:103C600004E00132019EFF0FFBD79951EF1601A02E
:103C700002D09A51EF1236EC12F09A51EF12982BB3
:103C8000E7D7120EE95E49EC11F049EC11F0120091
:103C900096C401F0010E006E015004E00036009061
:103CA000FF0FFBD700C09AF4001C0401996F986BBA
:103CB00094C4E9FF95C4EAFF976B9751070824E382
:103CC0009951EF16120EE9269951EF16EBEC10F010
:103CD0009A51EF12EBEC10F0120EE95E9A51EF14CC
:103CE000006E0CE097C401F0010E006E015004E07C
:103CF00000360090FF0FFBD70050981349EC11F0ED
:103D000049EC11F0972BD9D798C400F01200010E9E
:103D100004019E6FE80EA26F640EA36F000EA46FE5
:103D200041EC12F094C4A2F4950E0401A36F040EAA
:103D3000A46FAFEC10F0950EA26F040EA36F50ECC1
:103D400011F0E80EA26F650EA36F000EA46F41EC98
:103D500012F08D0E0401A26F650EA36F000EA46F0A
:103D600041EC12F0A0EC01F094C4C4F4F6EC01F0C4
:103D700000C09EF40050000A0CE0160E0401A26F71
:103D8000650EA36F000EA46F41EC12F004019E6B50
:103D90000CD004015E0EA26F650EA36F000EA46F1F
:103DA00041EC12F0010E04019E6F74EC02F03EEC47
:103DB00011F09EC400F012000301846B856B000EAD
:103DC000855D02E1FF0E845D16E28F0E8425E16EB3
:103DD000000E8521E26EE1CFE1FFE2CFE2FFE66A6D
:103DE000010E8425006E000E8521016E00C084F353
:103DF00001C085F3E4D7846B856B000E855D02E11D
:103E0000600E845D16E2170E8425E16E040E852196
:103E1000E26EE1CFE1FFE2CFE2FFE66A010E842528
:103E2000006E000E8521016E00C084F301C085F391
:103E3000E4D7846B856B000E855D02E1600E845DC6
:103E400016E29F0E8425E16E030E8521E26EE1CF1E
:103E5000E1FFE2CFE2FFE66A010E8425006E000E6C
:103E60008521016E00C084F301C085F3E4D78E0E76
:103E70000401A26F030EA36F3E0EA46F660EA56F22
:103E8000000EA66FC6EC11F0780E0401A26F040EAE
:103E9000A36F420EA46F660EA56F000EA66FC6EC50
:103EA00011F0070E0401A26F040EA36F460EA46F5B
:103EB000660EA56F000EA66FC6EC11F00301866BAF
:103EC000876B846B856BA4AA02D0AACF88F3886B1A
:103ED00000018D6B8E6BA38A2E6A2F6A1200000E72
:103EE0000401951902E1000E941937E094C4E9FF2A
:103EF00095C4EAFFEE5231E096C4A2F497C4A3F44D
:103F0000BEEC0EF000C0A6F494C4A2F495C4A3F4D1
:103F100096C4A4F497C4A5F43BEC0FF0000E01186E
:103F200002E1000E001805E194C400F095C401F010
:103F300016D0010E04019425A26F000E9521A36FE7
:103F400096C4E9FF97C4EAFFEECFA4F49DEC11F00C
:103F500000C094F401C095F4C2D7006A016A12004F
:103F6000620E0301246F020E256F000E266F000EF5
:103F7000276F400E286F030E296F000E2A6F000E68
:103F80002B6FFF0E2C6FFF0E2D6F000E2E6F000E8D
:103F90002F6FFF0E346FFF0E356FFF0E366FFF0E63
:103FA000376FEC0E446F030E456FC40E466F040E60
:103FB000476FE80E486F040E496F000E4A6F000EFF
:103FC0004B6F959295908C928C9095829580739E74
:103FD000739C380E726E120000C01BF001C01AF004
:103FE000E1CF1CF0E2CF1DF0A4AA92D0A3AA90D0FA
:103FF000AACF88F39CA202D09C989C889CA404D051
:10400000AACF88F30301886B03018551000802E100
:104010008451FF081BE284C386F385C387F3AACFCC
:1040200088F3886B8F0E8425E16E000E8521E26E89
:10403000E1CFE1FFE2CFE2FFE66A846B856B010E20
:1040400000018D6F000E8E6FA39A62D049D00301DC
:104050008851520A04E1010E2E6E000E2F6E58D0C8
:10406000030188514D0A04E1020E2E6E000E2F6EE0
:104070004FD003018851430A04E1030E2E6E000E57
:104080002F6E240E00018F6F470E906F500E916FB0
:10409000520E926F4D0E936F430E946F050E0301F7
:1040A000846F000E856F34D003018F0E8425E16E7E
:1040B000000E8521E26EE1CFE1FFE2CFE2FF88C38F
:1040C000E6FF84C386F385C387F3010E8425006E63
:1040D000000E8521016E00C084F301C085F318D065
:1040E000000E2F1802E1000E2E18B1E0000E2F185E
:1040F00002E1010E2E18B4E0000E2F1802E1020EAC
:104100002E18B7E0000E2F1802E1030E2E18CCE097
:104110009EAA50D09DAA4ED0AFCF21F3ACA203D01F
:10412000AC98AC88AC92ACA402D0AFCF21F3030121
:1041300021510D0A09E0000E006E8151005C02E180
:1041400080513F0801E31CD0010E0101936F000E66
:10415000946F9D9A170E03018025E16E020E812156
:10416000E26EE1CFE1FFE2CFE2FFE66A80C382F3D5
:1041700081C383F3806B816BAFCF21F3216B1AD0A6
:10418000170E8025E16E020E8121E26EE1CFE1FF84
:10419000E2CFE2FF21C3E6FF80C382F381C383F352
:1041A000010E8025006E000E8121016E00C080F39B
:1041B00001C081F31BC000F01AC001F01CC0E1FF78
:1041C0001DC0E2FF110000C019F001C018F0156E0B
:1041D000D8CF16F0E0CF17F0F2AA1DD0F2A41BD072
:1041E0006D0ED76E840ED66E010E245C006E000E2E
:1041F0002558016E00C024F001C025F0800E25185E
:10420000006E800E005C02E1010E245C03E20101FD
:104210009283F29AF2941750E06E1650D86E153AC7
:10422000153819C000F018C001F0100025EC33F06B
:10423000EDEC17F0010E1F6E89908992970E010127
:10424000956F010E966F8980948E949C959C958AAB
:104250009EEC17F000C091F10050040A03E1010147
:10426000928D02D00101929D7E86040E7F6EE10E3A
:10427000B06EAD8421EC19F0070E0B6E170E0C6EAC
:104280006A0E0D6E0D2EFED70C2EFCD70B2EFAD714
:1042900000007C86040E7D6EE10EAB6EA88400ECFF
:1042A00018F02AEC18F02BEC12F0950E0401A26F16
:1042B000630EA36F000EA46FEFEC11F03D0E04012E
:1042C000A26F610EA36F000EA46FEFEC11F0300E21
:1042D000010191250401CA6F0EEC00F0010191511A
:1042E000040A0AE1B00E0401A26F650EA36F000E6E
:1042F000A46FEFEC11F009D03E0E0401A26F650E21
:10430000A36F000EA46FEFEC11F02BEC12F0A39A48
:104310009D9AF28CD08E1F0E0B6E710E0C6E1E0EBF
:104320000D6E0D2EFED70C2EFCD70B2EFAD70000EB
:10433000898282EC14F08A980D0E0B6E2D0E0C6E95
:10434000D70E0D6E0D2EFED70C2EFCD70B2EFAD7E6
:1043500000000000F28EF80E0401A26F640EA36F3D
:10436000000EA46F41EC12F0070E0401A26F650E5F
:10437000A36F000EA46FEFEC11F0230E0401A26FE7
:10438000660EA36F000EA46FEFEC11F0290E04016E
:10439000A26F660EA36F000EA46F41EC12F00D0E1B
:1043A0000B6E2D0E0C6ED70E0D6E0D2EFED70C2E35
:1043B000FCD70B2EFAD700000000000E0101941963
:1043C00002E1010E931912E1C20E0401A26F620E06
:1043D000A36F000EA46F41EC12F0170E0401A26F40
:1043E000020EA36F50EC11F03EEC11F082EC14F0D1
:1043F000720E0401A26F650EA36F000EA46FEFECA6
:1044000011F0840E0401A26F650EA36F000EA46F5D
:1044100041EC12F0310E0B6EB40E0C6E650E0D6E8B
:104420000D2EFED70C2EFCD70B2EFAD70000000065
:10443000000E0101941902E1010E931912E1DC0E44
:104440000401A26F620EA36F000EA46F41EC12F084
:10445000170E0401A26F020EA36F50EC11F03EEC98
:1044600011F08A881F0E0B6E710E0C6E1E0E0D6EF3
:104470000D2EFED70C2EFCD70B2EFAD700003EECEB
:1044800011F0B00E0401A26F610EA36F000EA46FB5
:1044900041EC12F090EC17F003011F6B206B800EC3
:1044A0000401946F0F0E956F020E966F2FEC17F0AC
:1044B0004DEC19F0800E946F0F0E956F020E966FF3
:1044C000330E976F0FEC1EF04DEC19F0800E946FC9
:1044D0000F0E956F020E966F48EC1EF000C021F390
:1044E0004DEC19F0C80EA26F640EA36F000EA46FFE
:1044F00041EC12F003019F6B21C394F49F0E040161
:10450000956F030E966F08EC1DF09F0EA26F030EC1
:10451000A36F50EC11F0D80EA26F650EA36F000EC2
:10452000A46F41EC12F0C80E0401A26F650EA36FD8
:10453000000EA46FEFEC11F00301226B236B000E51
:10454000235D02E1060E225D34E2800E0401946FC9
:104550000F0E956F020E966F48EC1EF000C021F30F
:104560004DEC19F0170E03012225E16E030E2321F5
:10457000E26EE1CFE1FFE2CFE2FF21C3E6FF9F6BF6
:1045800021C394F49F0E0401956F030E966F08ECFF
:104590001DF09F0EA26F030EA36F50EC11F09F0E43
:1045A000A26F030EA36F10EC12F00301224B232B1A
:1045B000C6D7E00E0401A26F650EA36F000EA46FB4
:1045C00041EC12F0B80E0401A26F650EA36F000E4D
:1045D000A46FEFEC11F0800E0401946F0F0E956F35
:1045E000020E966F48EC1EF000C021F303019F6B92
:1045F00021C394F49F0E0401956F030E966F08EC8F
:104600001DF09F0EA26F030EA36F50EC11F03EEC55
:1046100011F09F0E0401A26F030EA36F10EC12F0B5
:104620002BEC12F0B60E0401A26F640EA36F000E05
:10463000A46FEFEC11F0A40E0401A26F640EA36F3F
:10464000000EA46F41EC12F0800E0401946F0F0E67
:10465000956F020E966F2FEC17F0800E946F0F0E71
:10466000956F020E966FCC0E976F0FEC1EF0800EBA
:10467000946F0F0E956F020E966F440E976F0FECAE
:104680001EF04DEC19F0800E946F0F0E956F020E18
:10469000966F2FEC17F0800E946F0F0E956F020E31
:1046A000966FCC0E976F0FEC1EF0800E946F0F0E6E
:1046B000956F020E966FBE0E976F0FEC1EF0250ED3
:1046C0000B6E870E0C6E8B0E0D6E0D2EFED70C2E04
:1046D000FCD70B2EFAD700000000800E946F0F0E4F
:1046E000956F020E966F48EC1EF000C020F0000E91
:1046F000216E800E946F0F0E956F020E966F48EC30
:104700001EF000C003F0026A20500224006E215007
:104710000320016E00C022F001C023F000C094F419
:1047200001C095F448EC1DF09F0EA26F030EA36F1D
:104730007BEC0FF09F0EA26F030EA36FBEEC0EF08A
:1047400000C064F001C065F09F0E0024A26F030E4C
:104750000120A36F7B0EA46F650EA56F000EA66FE0
:10476000C6EC11F09F0E0401A26F030EA36F50EC74
:1047700011F03EEC11F09F0E0401A26F030EA36F27
:1047800010EC12F02BEC12F03EEC11F0650E04016F
:10479000A26F610EA36F000EA46FEFEC11F0530E29
:1047A0000401A26F630EA36F000EA46F41EC12F020
:1047B000780E746EB0EC1FF031EC01F00050000A7E
:1047C00001E1FAD7070E0B6E170E0C6E6A0E0D6E16
:1047D0000D2EFED70C2EFCD70B2EFAD70000780E2C
:1047E0000001666F780E0401946F87EC1EF000C024
:1047F00064F0000E0001656F740E0301226F000E5D
:10480000236F000E235D02E1820E225D25E222C3AA
:1048100094F487EC1EF000C064F0000E0001656F98
:10482000070E0B6E170E0C6E6A0E0D6E0D2EFED758
:104830000C2EFCD70B2EFAD70000000E006E65512F
:10484000005C02E16451000801E206D0020E03019F
:104850002227000E2323D5D7070E0B6E170E0C6EE2
:104860006A0E0D6E0D2EFED70C2EFCD70B2EFAD72E
:104870000000000E0001651902E1000E64190DE14F
:104880000F0E0401A26F630EA36F000EA46F41EC24
:1048900012F089828990DAEF29F0920E0401A26F5A
:1048A000640EA36F000EA46FEFEC11F0310E040143
:1048B000A26F650EA36F000EA46F41EC12F0B9EC6D
:1048C00019F0070E0B6E170E0C6E6A0E0D6E0D2E84
:1048D000FED70C2EFCD70B2EFAD70000490E040190
:1048E000A26F650EA36F000EA46F41EC12F08FEC67
:1048F0001AF0070E0B6E170E0C6E6A0E0D6E0D2E53
:10490000FED70C2EFCD70B2EFAD70000FE0E0001AE
:10491000676FFF0E686F970E0101956F010E966F1E
:1049200083A601D0CBD1F28E57EC19F095C1A2F439
:1049300096C1A3F43D0E0401A46F630EA56F000E93
:10494000A66FC6EC11F00401946B956B95C196F4BB
:1049500096C197F4010E986FAEEC1AF095C1A2F4CF
:1049600096C1A3F450EC11F03EEC11F09FEC1AF05C
:104970009FEC1AF09FEC1AF095C1A2F496C1A3F433
:10498000400E0401A46F640EA56F000EA66FC6EC66
:1049900011F095C1A2F496C1A3F450EC11F03EECD5
:1049A00011F0010E0401946F010E956F95C196F4FC
:1049B00096C197F4010E986FAEEC1AF0140E946F36
:1049C000000E956F8EEC1CF057EC19F095C1A2F417
:1049D00096C1A3F4270E0401A46F630EA56F000E09
:1049E000A66FC6EC11F095C1A2F496C1A3F450ECE9
:1049F00011F03EEC11F00401946B956B95C196F4A7
:104A000096C197F4010E986FAEEC1AF095C1A2F41E
:104A100096C1A3F4650EA46F5D0EA56F000EA66F80
:104A2000C6EC11F0010E0401946F010E956F95C153
:104A300096F496C197F4010E986FAEEC1AF0140E2E
:104A4000946F000E956F8EEC1CF057EC19F095C129
:104A5000A2F496C1A3F47E0E0401A46F640EA56FA8
:104A6000000EA66FC6EC11F095C1A2F496C1A3F496
:104A700050EC11F03EEC11F00401946B956B95C174
:104A800096F496C197F4010E986FAEEC1AF095C1AA
:104A9000A2F496C1A3F4550EA46F640EA56F000E88
:104AA000A66FC6EC11F0010E0401946F030E956F12
:104AB00095C196F496C197F4010E986FAEEC1AF07A
:104AC000140E946F000E956F8EEC1CF057EC19F0DD
:104AD00095C1A2F496C1A3F4EC0E0401A46F630E79
:104AE000A56F000EA66FC6EC11F095C1A2F496C199
:104AF000A3F450EC11F03EEC11F00401946B956BB3
:104B000095C196F496C197F4010E986FAEEC1AF029
:104B100095C1A2F496C1A3F4D70EA46F630EA56F3E
:104B2000000EA66FC6EC11F0010E0401946F010E89
:104B3000956F95C196F496C197F4020E986FAEECFE
:104B40001AF0140E946F000E956F8EEC1CF057EC5B
:104B500019F0040E0B6E0C0E0C6E330E0D6E0D2E36
:104B6000FED70C2EFCD70B2EFAD70000000095C103
:104B7000A2F496C1A3F4160E0401A46F640EA56FEF
:104B8000000EA66FC6EC11F095C1A2F496C1A3F475
:104B900050EC11F0946B956B95C196F496C197F417
:104BA000010E986FAEEC1AF095C1A2F496C1A3F471
:104BB000070EA46F660EA56F000EA66FC6EC11F06F
:104BC00095C1A2F496C1A3F450EC11F03EEC11F0A3
:104BD000010E0401946F010E956F95C196F496C174
:104BE00097F4030E986FAEEC1AF0140E946F000E4B
:104BF000956F8EEC1CF057EC19F0040E0B6E0C0E3A
:104C00000C6E330E0D6E0D2EFED70C2EFCD70B2E18
:104C1000FAD70000000095C1A2F496C1A3F4F60EE5
:104C20000401A46F620EA56F000EA66FC6EC11F012
:104C300095C1A2F496C1A3F450EC11F0080E946F44
:104C4000010E956F030E966F2CEC1CF0100E946FF6
:104C5000010E956F010E966F2CEC1CF0200E946FD8
:104C6000010E956F020E966F2CEC1CF0140E946FD3
:104C7000000E956F8EEC1CF057EC19F095C1A2F464
:104C800096C1A3F42B0E0401A46F640EA56F000E51
:104C9000A66FC6EC11F095C1A2F496C1A3F450EC36
:104CA00011F03EEC11F0FF0E0401946F5DEC17F073
:104CB000140E946F000E956F8EEC1CF057EC19F0EB
:104CC000F28CF28CF28E898089928970800E0401B8
:104CD000946F0F0E956F020E966F2FEC17F0800EEB
:104CE000946F0F0E956F020E966FCC0E976F0FECB0
:104CF0001EF0800E946F0F0E956F020E966F440E8D
:104D0000976F0FEC1EF04DEC19F0800E946F0F0EA4
:104D1000956F020E966F2FEC17F0800E946F0F0EAA
:104D2000956F020E966FCC0E976F0FEC1EF0800EF3
:104D3000946F0F0E956F020E966FBE0E976F0FEC6D
:104D40001EF0130E0B6E440E0C6E440E0D6E0D2EE7
:104D5000FED70C2EFCD70B2EFAD70000800E946FD6
:104D60000F0E956F020E966F48EC1EF000C020F0FB
:104D7000000E216E800E946F0F0E956F020E966FCF
:104D800048EC1EF000C003F0026A20500224006EBE
:104D900021500320016E00C022F001C023F000C0AA
:104DA00094F401C095F448EC1DF000C061F09F0E32
:104DB000A26F030EA36F7BEC0FF09F0EA26F030E8A
:104DC000A36FBEEC0EF000C064F001C065F0020EEF
:104DD000005C026E000E0158036E9F0E0224E96E05
:104DE000030E0320EA6EE9CFE9FFEACFEAFF300EB7
:104DF000EE5C036E03C004F00436049004360490A5
:104E00000436049004360490010E005C026E000E1D
:104E10000158036E9F0E0224E96E030E0320EA6E12
:104E2000E9CFE9FFEACFEAFF300EEE5C026E0250F6
:104E300004240001626F050E005C026E000E015832
:104E4000036E9F0E0224E96E030E0320EA6EE9CF83
:104E5000E9FFEACFEAFF300EEE5C046E04C002F018
:104E6000023602900236029002360290023602901A
:104E7000040E005E000E015A9F0E0024E96E030E20
:104E80000120EA6EE9CFE9FFEACFEAFF300EEE5CDF
:104E9000006E00500224636F690E0401A26F000EC1
:104EA000A36F6A0EA46F640EA56F000EA66FC6EC0A
:104EB00011F0720E0401946F000E956F9F0E966FA5
:104EC000030E976F010E0001645D0401986F000EE0
:104ED000000165590401996FC4EC1CF0690EA26FC2
:104EE000000EA36F50EC11F0270E0001786F090E31
:104EF0000401CA6F15EC00F08E0E0401A26F030EC0
:104F0000A36F390EA46F660EA56F000EA66FC6ECD8
:104F100011F0780E0401A26F040EA36F2F0EA46F80
:104F2000660EA56F000EA66FC6EC11F0070E040109
:104F3000A26F040EA36F340EA46F660EA56F000E51
:104F4000A66FC6EC11F0DCEC1EF0350E0401A26F6A
:104F5000620EA36F000EA46F41EC12F08972430E33
:104F60000B6EF70E0C6EAD0E0D6E0D2EFED70C2EC9
:104F7000FCD70B2EFAD7000E00018E1902E1010EAC
:104F80008D19D8A498D00101406BF29A83B61DD038
:104F900083B41BD0D30E0401A26F610EA36F000E69
:104FA000A46F41EC12F08F0E0401A26F000EA36FEC
:104FB00050EC11F03EEC11F08F0E0401A26F000EC8
:104FC000A36F10EC12F02BEC12F09F0E0401A26FF5
:104FD000030EA36F000EA46F660EA56F000EA66FE2
:104FE000C6EC11F08F0E0401946F000E956F9F0EAA
:104FF000966F030E976F6FEC1FF000C08FF101C02A
:1050000090F1000E026E0150025C02E100500008B7
:1050100051E20301226B236B000E235D02E15F0E60
:10502000225D1DE2170E2225E16E040E2321E26EA1
:10503000225101018F25E96E0301235101019021C5
:10504000EA6EE9CFE9FFEACFEAFFE1CFE1FFE2CF85
:10505000E2FFEECFE6FF0301224B232BDDD75F0EED
:1050600001018F25E16E000E9021E26EE1CFE1FF9C
:10507000E2CFE2FFE66A62EC12F000C01EF00050E0
:105080000A0A18E1AFEC14F08A0E0401946F030EC3
:10509000956FB6EC18F000C087F001C088F01F5083
:1050A000000A08E1A80EA26F650EA36F000EA46FA0
:1050B00041EC12F012D0F40E0401A26F610EA36F46
:1050C000000EA46F41EC12F0A80E0401A26F620E54
:1050D000A36F000EA46FEFEC11F0970E0101956F16
:1050E000010E966F010E00016715016E68C002F097
:1050F000000E0216000E021802E1000E011829E14E
:1051000095C1A2F496C1A3F4010E0401A46F640E2C
:10511000A56F000EA66FC6EC11F067C0A2F468C0C0
:10512000A3F40C0E010195250401A46F000E0101EA
:1051300096210401A56FF0EC0EF0010E946F956BB3
:1051400095C196F496C197F4010E986FAEEC1AF0E3
:105150000CD00401010E946F956B690E966F000ED2
:10516000976F010E986FAEEC1AF0970E0101956FD4
:10517000010E966F95C1A2F496C1A3F4C10E04016D
:10518000A46F630EA56F000EA66FC6EC11F0070E9C
:10519000010195250401A26F000E01019621040171
:1051A000A36F8E0EA46F030EA56F76EC11F095C160
:1051B000A2F496C1A3F4BEEC0EF000C064F001C0EE
:1051C00065F0000E015C02E1140E005C10E20001CB
:1051D000645101019525E16E00016551010196219F
:1051E000E26EE1CFE1FFE2CFE2FF200EE66E010EBC
:1051F0000401946F010E956F95C196F496C197F4D2
:10520000010E986FAEEC1AF0970E0101956F010E2A
:10521000966F95C1A2F496C1A3F4AB0E0401A46FDE
:10522000630EA56F000EA66FC6EC11F0070E01010C
:1052300095250401A26F000E010196210401A36FC0
:10524000780EA46F040EA56F76EC11F095C1A2F450
:1052500096C1A3F4BEEC0EF000C064F001C065F08E
:10526000000E015C02E1140E005C10E200016451CA
:1052700001019525E16E0001655101019621E26E63
:10528000E1CFE1FFE2CFE2FF200EE66E010E040166
:10529000946F020E956F95C196F496C197F4010E26
:1052A000986FAEEC1AF0970E0101956F010E966F94
:1052B00095C1A2F496C1A3F4690E0401A46F630E14
:1052C000A56F000EA66FC6EC11F0070E0101952523
:1052D0000401A26F000E010196210401A36F070EC5
:1052E000A46F040EA56F76EC11F095C1A2F496C1DF
:1052F000A3F4BEEC0EF000C064F001C065F0000E37
:10530000015C02E1140E005C10E200016451010135
:105310009525E16E0001655101019621E26EE1CF14
:10532000E1FFE2CFE2FF200EE66E010E0401946F72
:10533000030E956F95C196F496C197F4010E986F80
:10534000AEEC1AF00001674B682B83B604D083A43F
:1053500002D0010E1F6E83B402D083B61F6A82ECA6
:1053600014F03D0E0B6EE10E0C6E3F0E0D6E0D2E09
:10537000FED70C2EFCD70B2EFAD700000000000E33
:10538000941902E1010E931914E1BA0E0401A26FFF
:10539000600EA36F000EA46F41EC12F00201576B78
:1053A000170E0401A26F020EA36F50EC11F03EEC39
:1053B00011F08BD4FFD700000000000000000000B7
:1053C000000000000000000000F8000000000000E5
:1053D00000333000000000100C06100C0600000026
:1053E00000000000000040C07840C0784000043F4A
:1053F00004043F040400007088FC0830000000181A
:1054000020FF211E0000F008F000E018000000213D
:105410001C031E211E0000F00888700000001E21E1
:1054200023241927211010160E0000000000000090
:10543000000000000000000000E01804020000006E
:1054400000071820400000020418E000000000409F
:10545000201807000000404080F080404000020219
:10546000010F01020200000000F000000000010135
:10547000011F01010100000000000000000080B0D9
:1054800070000000000000000000000000000001AB
:1054900001010101010100000000000000000030D6
:1054A0003000000000000000000080601804006070
:1054B00018060100000000E010080810E000000FCE
:1054C000102020100F00001010F800000000002035
:1054D000203F20200000007008080888700000307D
:1054E0002824222130000030088888483000001825
:1054F000202020110E000000C02010F8000000073E
:105500000424243F240000F80888880808000019B3
:10551000212020110E0000E0108888180000000FE4
:10552000112020110E0000380808C83808000000BB
:10553000003F000000000070880808887000001C10
:10554000222121221C0000E010080810E0000000C9
:10555000312222110F00000000C0C0000000000036
:10556000003030000000000000800000000000005B
:105570008060000000000000804020100800000152
:105580000204081020004040404040404000040415
:1055900004040404040000081020408000000020DF
:1055A000100804020100007048080808F00000001C
:1055B000003036010000C030C828E810E0000718AD
:1055C000272423140B000000C038E0000000203C1A
:1055D00023020227382008F8888888700000203FBE
:1055E000202020110E00C0300808080838000718D5
:1055F00020202010080008F808080810E000203FCC
:10560000202020100F0008F88888E8081000203FAC
:1056100020202320180008F88888E8081000203F80
:10562000200003000000C0300808083800000718F8
:105630002020221E020008F808000008F808203F79
:10564000210101213F20000808F80808000000207F
:10565000203F2020000000000808F8080800C08053
:1056600080807F00000008F888C028180800203FCC
:1056700020012638200008F8080000000000203F24
:1056800020202020300008F8F800F8F80800203F1B
:10569000003F003F200008F830C00008F808203F15
:1056A000200007183F00E01008080810E0000F1065
:1056B000202020100F0008F808080808F000203FFC
:1056C000210101010000E01008080810E0000F1897
:1056D000242438504F0008F8888888887000203FBC
:1056E0002000030C302000708808080838000038BB
:1056F000202121221C00180808F8080818000000C2
:10570000203F2000000008F808000008F808001FEB
:10571000202020201F000878880000C838080000DA
:1057200007380E010000F80800F80008F800033CF4
:105730000700073C030008186880806818082030BC
:105740002C03032C30200838C800C838080000009B
:10575000203F2000000010080808C8380800203842
:10576000262120201800000000FE02020200000096
:10577000007F40404000000C30C0000000000000EE
:1057800000010638C00000020202FE0000000040D6
:1057900040407F00000000000402020204000000FC
:1057A00000000000000000000000000000008080F9
:1057B00080808080808000020204000000000000E1
:1057C00000000000000000008080808000000019C0
:1057D000242222223F2008F8008080000000003FA1
:1057E000112020110E000000008080800000000EBB
:1057F000112020201100000000808088F800000E99
:10580000112020103F200000808080800000001FB9
:10581000222222221300008080F08888881800202D
:10582000203F202000000000808080808000006BEE
:1058300094949493600008F8008080800000203FDA
:10584000210000203F2000809898000000000020E8
:10585000203F20200000000000809898000000C039
:105860008080807F000008F8000080808000203F5A
:1058700024022D302000000808F80000000000205D
:10588000203F202000008080808080808000203F9A
:1058900020003F20003F8080008080800000203F6B
:1058A000210000203F200000808080800000001F39
:1058B000202020201F00808000808000000080FFCA
:1058C000A12020110E000000008080808000000ECA
:1058D000112020A0FF808080800080808000202018
:1058E0003F21200001000000808080808000003384
:1058F000242424241900008080E08080000000001F
:10590000001F202000008080000000808000001F19
:10591000202020103F2080808000008080800001B7
:105920000E300806010080800080008080800F30EB
:105930000C030C300F00008080008080800000206D
:10594000312E0E3120008080800000808080808198
:105950008E70180601000080808080808000002109
:10596000302C2221300000000000807C0202000068
:105970000000003F404000000000FF000000000069
:105980000000FF0000000002027C800000000040D8
:10599000403F000000000006010102020404000074
:1059A0000000000000000000000000000000002FC8
:1059B000000000000700070000147F147F1400247B
:1059C0002A7F2A12006264081323003649552250A8
:1059D0000F090F09000000001C22410000004122B5
:1059E0001C000014083E08140008083E08080000C7
:1059F00000A06000000808080808000060600000BF
:105A0000002010080402003E5149453E0000427F3C
:105A10004000004261514946002141454B31001888
:105A200014127F10002745454539003C4A4949304A
:105A30000001710905030036494949360006494904
:105A4000291E00003636000000005636000000080F
:105A500014224100001414141414000041221408EC
:105A600000020151090600324959513E007C1211D1
:105A7000127C007F49494936003E41414122007F66
:105A80004141221C007F49494941007F0909090120
:105A9000003E4149497A007F0808087F0000417FA5
:105AA0004100002040413F01007F08142241007F57
:105AB00040404040007F020C027F007F0408107FBE
:105AC000003E4141413E007F09090906003E415127
:105AD000215E007F091929460046494949310001E4
:105AE000017F0101003F4040403F001F2040201F38
:105AF000003F4038403F00631408146300070870FB
:105B0000080700615149454300007F414100000200
:105B100004081020000041417F000004020102043B
:105B20000040404040400000010204000020545466
:105B30005478007F484444380038444444200038B6
:105B40004444487F00385454541800087E09010228
:105B50000018A4A4A47C007F080404780000447DFD
:105B60004000004080847D00007F10284400000039
:105B7000417F4000007C04180478007C080404780D
:105B800000384444443800FC2424241800182424F9
:105B900018FC007C080404080048545454200004F5
:105BA0003F444020003C4040207C001C2040201C02
:105BB000003C4030403C004428102844001CA0A079
:105BC000A07C004464544C4414141414141420484D
:105BD000617264773A202050494320436C69636BBB
:105BE00065722031384634374A3533200D0A204F4C
:105BF0006C65642053534431333036203132387869
:105C0000333220302E3936200D0A204453313842A9
:105C100032302073656E736F72200D0A2047505327
:105C20002055426C6F7820374E200D0A2055415286
:105C30005432200D0A0D0A0020446F737369657297
:105C40003A433A5C5F4D696B726F435C5F436C69CA
:105C5000636B65725F31384634374A35335F47507E
:105C600053374E5F747261636B65725F4F6C65642E
:105C70005F445331384232305F55415254735F3282
:105C80003032350D0A0020536F75726365203A205B
:105C90005F436C69636B65725F31384634374A35F0
:105CA000335F475053374E5F747261636B65725F49
:105CB0004F6C65645F445331384232305F55415216
:105CC00054735F5F323032352D303630362E630DEF
:105CD0000A0020417574726573203A20204F4C45AC
:105CE000445F493243325F3139303830312E6320DE
:105CF0002C204F4C45445F4932435F3139303830B6
:105D0000312E68202C204F4C45445F5461626C65F5
:105D1000735F313930382E680D0A0D0A0020507239
:105D20006F6A65743A5F436C69636B65725F3138A3
:105D30004634374A35335F475053374E5F7472618C
:105D4000636B65725F4F6C65645F445331384232F8
:105D5000305F55415254735F323032352E6D63706F
:105D600070690D0A0033206C69676E657320646585
:105D700020323020636172732041424344454647DC
:105D800048494A4B4C4D4E4F50515253545556571B
:105D900058595A206162636465666768696A6B6C0A
:105DA0006D6E6F70717273747576777800205541DF
:105DB00052543120666F722048433132206D617039
:105DC00070656420393630302C382C4E2C312054FC
:105DD000582070696E205244362D52503232202C99
:105DE0002052782070696E205244352D5250323343
:105DF0000D0A000000000000000600000000002C5A
:105E0000002C00000000000000F065001C6600157A
:105E10006600C06500AA5E00DA5E006A5F009A5FF5
:105E2000000A5F003A5F008A60005A6000CA5F00A3
:105E3000FA5F002A600020496E666F732061666613
:105E4000696368E965732076696120554152543170
:105E5000206D6F64756CE9657320656E20666F6EEA
:105E60006374696F6E206465204250312065742030
:105E70004250320D0A0020554152543220666F7252
:105E80002047505320393630302C382C4E2C3120BE
:105E900054582070696E20524336202C20527820AE
:105EA00070696E205243370D0A000080F0FCFEFE40
:105EB0003F0F0F0F3FFEFEFCF08000FFFFFFFFFFD4
:105EC0000000000000FFFFFFFFFF00030F3F7F7F88
:105ED000FCF0F0F0FC7F7F3F0F01000000C0E0E02D
:105EE000F0F87CFEFFFFFFFF00000000000301014F
:105EF000000000FFFFFFFFFF0000000000000000A7
:105F0000000000FFFFFFFFFF00000000000000C0D6
:105F1000E0F8FCFFFFFFFFFF0000C0E0F8FCFFBF60
:105F20008F8381FFFFFFFFFF8080070707070707B9
:105F3000070707FFFFFFFFFF0707000080FCFFFFC9
:105F4000FF3F1F1F1F1F1F1F1F0000183F3F3F3F26
:105F50001F0F0F0F1FFFFEFEF8E000061F3F7F7FA1
:105F6000FCF0F0F0F87F7F3F1F0700E0F8FCFEFE3A
:105F70001F0F0F0F1FFFFEFEFCF00000000000804F
:105F8000C0E0F0F8FE7F3F1F070100C0F8FCFFFFF4
:105F9000FFFFF9F9F8F8F8F8F8F80030787E7E7F1E
:105FA0001F0F0F1FFFFEFEFCF000000000000000AE
:105FB000000E0E0F1FFBFBF9F0C000061F3F7F7F96
:105FC000FCF0F0F0FC7F7F3F1F0700F0FCFEFEFFBF
:105FD0001F0F0F0F1FFFFEFEFCF00081C3E7FFFF46
:105FE0007E3C3C3C7EFFFFE7C381000F3F7F7FFF8D
:105FF000F8F0F0F0F8FF7F7F3F0F00E0F8FCFEFFC5
:106000001F0F0F0F1FFEFEFCF08000070F3F3F7FAA
:106010007C7878783CFFFFFFFFFF000E3E7E7EFE1F
:10602000F8F0F0F07C7F3F1F0F010000000000003F
:106030000000000000000000000000000000000060
:106040000000000000000000000000000000000050
:1060500000000000FFFFFFFF0000001F1F1F1F1FA9
:106060001F1F1F9FFFFFFF3F1F0F0000000000E0EA
:10607000F8FCFF7F0F0300000000000000F0FFFFAE
:10608000FFFF07000000000000000080F0F8FCFEA9
:106090003E0F0F0F1F7F7E7E7C7000FFFFFFFFFF14
:1060A0003C1E1E1E3EFEFCFCF0E000010F3F7F7F09
:1060B000F8F0F0F0F8FF7F3F1F072052656375206E
:1060C000646520484331322064697374616E7420C2
:1060D00028554152543120525820E0203936303072
:1060E0007329203A0D0A002070696E205242342034
:1060F0006F7574707574203D3E2063646520534550
:106100005420286D6F646520415429204843313262
:106110000D0A00204275732049324320706F75725A
:1061200020456372616E204F4C45442053534431E7
:10613000333036203132387833320D0A0020526540
:10614000746F7572204D617070616765732070693E
:106150006E7320554152543120657420554152547C
:1061600032203D20002049324320696E6974202886
:106170004F4C454420646F697420657472652063D8
:106180006F6E6E656374652021290D0A000D0A4B40
:106190006579626F61726420546F75636820554140
:1061A000525431206F722054696D656F75742000F0
:1061B000205465737420536F6E6465204F575320CD
:1061C00044533138423230207375722052413220AC
:1061D0000D0A00526563657074696F6E2073757285
:1061E000205541525432205258203D2047505320D0
:1061F0003A0D0A002042414420526563657074697B
:106200006F6E206F75204465636F6461676520471A
:1062100047410D0A00206F752034206C69676E6558
:1062200073206465203230206361727320367838C1
:1062300070200D0A002055415254322C207761699C
:1062400074696E6720475053206461746173203A0B
:106250002000204D435520203A2031384634374A1B
:1062600035335F51464E5F343470696E0D0A00203D
:10627000524431202D2D3E2049324332202D2D3ED7
:10628000534441204F4C4544200D0A0020524430D5
:10629000202D2D3E2049324332202D3E2053434CA9
:1062A000204F4C45440D0A00204D6175766169739D
:1062B0006520526563657074696F6E204750530D99
:1062C0000A00205265746F7572206465204843315E
:1062D00032206C6F63616C203A0D0A0020526574A5
:1062E0006F75722064652048433132206C6F6361A2
:1062F0006C203A0D0A0020416666696368652033A8
:106300002063617273205370656369617578002042
:106310004F4C4544204C4344204E6F6E2074726FA6
:106320007576E9200D0A00426967204D7367206485
:10633000652036302063617273203A2000203230AD
:1063400020436861727320737572204C69676E65B3
:106350002031004932433220696E69742061742013
:106360003130304B687A0D0A0020416C74693A2054
:10637000202020202020202020202020202000203D
:10638000506F77657220737570706C793A20342E77
:1063900035560D0A0020496E69742055415254311A
:1063A00020393630306264730D0A00204C61746904
:1063B0003A202020202020202020202020202020C3
:1063C00000204C6F6E673A202020202020202020C3
:1063D0002020202020200031323334353637383920
:1063E0003031323334353637383930004D73672029
:1063F00031342063617273207461696C6C65203282
:106400000020426F75636C6520232020202020200F
:10641000202020202000203720204269672043616F
:106420007273202031367831362000204F6C65643D
:106430002046494C4C2077697468203078464600E5
:106440003132333435362D4142432D6162632D366E
:1064500037383930004C34204E554D424552532088
:10646000303132333435363738002054656D70653D
:10647000723D2020202020202064656743004D735A
:1064800067207375722034656D204C69676E6520D6
:1064900020000D0A204F4C45442074726F757665BC
:1064A000200D0A00204D6573757265204453313804
:1064B0004232303D2000204D657375726520445393
:1064C00031384232303D20002046616D696C7920C0
:1064D000436F6465203A200030313233343536372B
:1064E0003839414243444546436865636B204465FF
:1064F000766963652040200020436F6E66696720DF
:10650000484331320D0A0020436F6E6669672048A8
:106510004331320D0A00206973206E6F7420666F5C
:10652000756E64002078203130306D7365630D0A1C
:1065300000204F4C454420696E69740D0A00202EDE
:106540002E42414420210D0A00204F4C4544204F4B
:106550004E0D0A002C20536174656C3A20002066B1
:106560006F756E64204F4B002C2048444F50203AEA
:1065700020002041542B52580D0A002064656720EA
:10658000432020002041542B52580D0A0032202075
:106590004841524457002C204C6174203A20002C72
:1065A00020416C74203A20002E2E204F4B0D0A0003
:1065B000202E2E4F4B0D0A0020204352433D200039
:1065C0000F090F000000000020494431203D200049
:1065D000204C6F6E203A200020494431203D20009D
:1065E00020204352433D2000206F6E20493243005B
:1065F00000007E66667E00002C204669783A200006
:10660000244750474741003132342E3936004B4D34
:106610004C203A2000060C1C7C1C0C06C030383E76
:106620003830602041540D0A002041540D0A0030DA
:106630002E303000302E303000302E3030002058D8
:10664000200020592000205A200010EE1EF0430E9A
:10665000006E010E016EF30EF66E5D0EF76E000E0B
:10666000F86EE5EC17F01200FFFFFFFFFFFFFFFFE2
:020000040001F9
:08FFF800ACF7FCFFFFFBFFFB6F
:00000001FF
